:020000040800F2
:10000000E0100020050100082F3800080929000829
:100010002D380008350F00080161000800000000BD
:100020000000000000000000000000004947000838
:10003000BF1A000800000000A13D0008314A000876
:100040001F0100089D3B00081F0100081F01000858
:100050001F0100081F0100081F0100081F01000800
:100060001F0100081F0100081F0100081F010008F0
:100070001F0100081F010008811500081F0100086A
:100080001F0100081F010008410700081F010008A8
:100090001F0100081F0100081F0100081F010008C0
:1000A000A14A0008814B00081F0100081F01000839
:1000B000854B0008754E0008D15000081F0100084C
:1000C0001F0100081F0100081F0100081F01000890
:1000D0001F010008F95B00081F0100081F0100084C
:1000E0001F0100081F0100081F010008DFF810D0E1
:1000F00000F0E8FA0048004741720008AFF30080C2
:10010000E01000200648804706480047FEE7FEE76B
:10011000FEE7FEE7FEE7FEE7FEE7FEE7FEE7FEE7B7
:10012000514A0008ED0000082DE9F0410024061BAB
:10013000254671F1000605DA01240027D0EB0700FF
:1001400067EB0101161E73F1000605DA0027D2EBFA
:100150000702012567EB030300F0D0F986460E463F
:1001600017469C46AC4204D00025D0EB050E65EB4B
:10017000010624B10020D2EB000760EB030C7046AF
:1001800031463A466346BDE8F08140EA01039B07E9
:1001900003D009E008C9121F08C0042AFAD203E0FC
:1001A00011F8013B00F8013B521EF9D2704780EA7A
:1001B000010210B502F00043400022D04A001FD0D7
:1001C000010E01EB1261C0F35600C2F3560240F477
:1001D000000042F40002A0FB022000047F39140456
:1001E00000D0401C50EA124001D44000491EC2B267
:1001F0000C0604EBD010401C4008802A02D003E01B
:10020000002010BD20F00100002900DA0020184372
:1002100010BD2DE9FE4F81EA030404F0004421F0F3
:10022000004100944FF0000B23F0004350EA01041A
:100230005ED052EA03045BD0C3F30A54C1F30A55FB
:100240002C44A4F2F3340194A0FB0254C1F3130133
:1002500041F48011C3F3130343F4801301FB024400
:1002600000FB034E840A970A44EA815447EA835705
:10027000A4FB076802958D0A05FB07854FEA932CBE
:1002800004FB0C542705029D4FEA065847EA16372F
:10029000B5EB08056EEB070C870E920E47EA811747
:1002A00042EA8312A7FB0201B6EB0B0164EB0004E8
:1002B0002B0D43EA0C335E1844EB1C50DA465146D2
:1002C000E7FB0201C5F313044FEA0B3343EA14536F
:1002D0004FEA0432019C43EA0603A4F10C040294A1
:1002E000009CCDE900B400F09FF903B0BDE8F08FA9
:1002F00000200146F9E72DE9F04D81EA030404F0FE
:10030000004B21F0004514464FF0000A23F0004155
:1003100050EA050220D054EA01021DD0C5F30A5765
:100320000246C5F31303C1F31300C1F30A5640F4A8
:10033000801543F48013A7EB0608101BD64608F27D
:10034000FD3873EB050002D308F1010801E09218B3
:100350005B41B8F1000F03DA00200146BDE8F08DE3
:1003600000204FF48011064684460EE0171B73EB05
:10037000050705D3121B63EB050306434CEA010C8A
:1003800049084FEA300092185B4150EA0107EDD16D
:1003900052EA030012D082EA040083EA050108430E
:1003A00005D0101BAB4106D20122002306E000223B
:1003B0004FF0004302E06FF0010253101AEB060009
:1003C0004CEB085110EB0A0041EB0B01BDE8F04D7E
:1003D00000F01BB970B521F0004303430CD0C1F30A
:1003E0000A550024D5EB040564EB0403D617AD1AB7
:1003F000B34102DB0020014670BD201841EB0251E1
:1004000070BDC10F80EAE0700844CA07962300213E
:1004100000F0CDB896230022114600F0C8B80EB502
:10042000C10F80EAE0700844CA07002140F233435C
:100430008DE80E000A460B4600F0F6F803B000BD4A
:100440000EB540F2334102910021CDE900110A4678
:100450000B4600F0E9F803B000BD00F0004220F0C8
:100460000040C10DC0F3160040F400007F2901DAFE
:1004700000207047962903DCC1F19601C84001E0D5
:1004800096398840002AF4D04042704770B5C1F3D5
:100490000A5201F000450024C1F3130140F2FF337A
:1004A00041F480119A4201DA002070BD40F23343DA
:1004B0009A42A2F2334203DC524200F05FF800E0BD
:1004C00090402C43F1D0404270BDC1F30A5210B5A8
:1004D000C1F3130140F2FF3341F480119A4201DA73
:1004E000002010BD40F233439A42A2F2334203DCB3
:1004F000524200F043F810BD904010BD2DE9F05F6E
:100500000546002092469B46884606468146402482
:100510001BE0284641464746224600F02FF8534646
:100520005A46C01A914110D311461846224600F08F
:1005300016F82D1A67EB01084F46224601200021CC
:1005400000F00DF817EB00094E41201EA4F1010444
:10055000DFDC484631462A464346BDE8F09F202A64
:1005600004DB203A00FA02F1002070479140C2F10A
:10057000200320FA03F3194390407047202A04DB3C
:10058000203A21FA02F00021704721FA02F3D0400C
:10059000C2F1200291400843194670470029A8BFC4
:1005A0007047401C490008BF20F00100704710B49C
:1005B000B0FA80FC00FA0CF050EA010404BF10BC51
:1005C000704749B1CCF1200421FA04F411FA0CF17E
:1005D00018BF012121430843A3EB0C01CB1D4FEAB7
:1005E00000614FEA102042BF002010BC704700EBB2
:1005F000C35010440029A4BF10BC7047401C4900E0
:1006000008BF20F0010010BC704710B5141E73F134
:10061000000408DA401C41F1000192185B411A43C2
:1006200001D120F0010010BD2DE9F04D92469B460E
:1006300011B1B1FA81F202E0B0FA80F220329046B4
:10064000FFF78DFF04460F4640EA0A0041EA0B011E
:1006500053465A46084313D0114653EA010019D0B5
:10066000C8F140025046FFF789FF05460E46504646
:1006700059464246FFF773FF084305D0012004E0C6
:1006800020463946BDE8F08D0020054346EAE07675
:100690002C4337430A986305E40AA0EB08000022C4
:1006A000FD0A44EA47540A3002D500200146E9E732
:1006B000010510196941DDE9084500196941BDE8E6
:1006C000F04DA2E7064C074D06E0E06840F001035C
:1006D00094E8070098471034AC42F6D3FFF70AFDC0
:1006E000649600088496000870B58C1810F8015BB9
:1006F00015F0070301D110F8013B2A1106D110F8BB
:10070000012B03E010F8016B01F8016B5B1EF9D1BE
:100710002B0705D40023521E0DD401F8013BFAE744
:1007200010F8013BCB1A921C03E013F8015B01F8AF
:10073000015B521EF9D5A142D8D3002070BD000044
:1007400070B54E4C4FF490652946204600F019FADA
:10075000002864D02946204600F0A6F848490888B9
:10076000401C08800121204600F0EAFA454942F287
:100770001072B1F85000904202D2401CA1F8500013
:1007800006F03AFF404DB5F91410B5F9120005F026
:10079000F9FD3E4CA5F84E002080A1682046884710
:1007A000A088A5F8500003F0ABF807F027F8384E02
:1007B000384C3078082833D045F6AC30606042F6CB
:1007C000EF60A06042F2C400E0603348008A2080FD
:1007D000208E6080A16B2F488847208E69882F4C1F
:1007E00008444FF6FF7101EA80006886207A4FF0D6
:1007F000000540071DD501F0F1FA294949F6A2404C
:100800000880284840F21A62C188491C89B2C18018
:10081000914204D3A16821F00401A160C58070BD9C
:1008200041F2130060604FF48060A06040F61B50FE
:10083000CAE730780A281BD2DFE800F01A0616054E
:100840000A050D1A1114EAE7BDE8704005F03EBF35
:1008500008F01EF808E0BDE8704002F09BBD06F00D
:10086000C7FA01E007F022F9BDE8704007F01EB9B1
:1008700000F0F8FB84F8B65070BD00000024014081
:1008800004070020480100206C0000202007002001
:10089000FB060020DC000020F8010020A40200205C
:1008A000442C0140240900206FEA112101607047A7
:1008B0000029816802D041F0010101E021F001012D
:1008C000816070470029816802D041F4807101E0A5
:1008D00021F48071816070472DE9F041824E92B021
:1008E000304600F00BF90BA800F039FA01214FF463
:1008F000C06003F00BFB00248DF831404FF4602002
:10090000CDE90D044FF4A0204FF009080B9001270A
:100910008DF83C808DF830700BA9304600F080F9DE
:10092000724D8DF831408DF830708DF83C700BA908
:10093000284600F075F901231A460F21304600F0D1
:10094000C0F9022201231146304600F0BAF9012312
:1009500003220021304600F0B4F901230422194695
:10096000304600F0AEF9012305220B21304600F09D
:10097000A8F9012306220421304600F0A2F9012340
:1009800007220821304600F09CF9012308220321A8
:10099000304600F096F9012309220A21304600F082
:1009A00090F90121304600F084F90121284600F039
:1009B00080F901231A460521304600F055F901233C
:1009C0001A460621284600F04FF90021304600F073
:1009D000CBF84FF4E041284600F0C6F8012130463C
:1009E00000F0B8F80121284600F0B4F801213046A3
:1009F00000F0A6F80121284600F0A2F801213046B7
:100A000000F09EF90121284600F09AF940F61451B1
:100A1000374804F034FE12208DF8400002208DF893
:100A200041008DF842408DF8437010A802F02CFF71
:100A300001224FF49061304600F0E8F80121304681
:100A4000FFF740FF01213046FFF732FF0121284622
:100A5000FFF72EFF304600F06EF9304600F09FF8A9
:100A60000028FAD1304600F075F9304600F082F8DF
:100A70000028FAD1284600F05EF9284600F08FF8E9
:100A80000028FAD1284600F065F9284600F072F8EF
:100A90000028FAD10121084603F014FA154D284622
:100AA00000F0AAFD684600F052FE0F4801A94C3044
:100AB0000090114881E811018020CDE904404000F8
:100AC000069080000790202008904FF44050CDE918
:100AD00009046946284600F01DFE0121284600F061
:100AE0007FFD12B0BDE8F0810024014000280140E4
:100AF000002C014008000240B40200200D4910B54E
:100B0000884202D1012144150AE00B49884202D1F2
:100B10000121041504E0094988420AD10121CC03CE
:100B2000204603F0FFF92046BDE81040002103F005
:100B3000F9B910BD0024014000280140003C0140EB
:100B40000029816802D041F4801101E021F4801174
:100B5000816070470029816802D041F4004101E0C2
:100B600021F4004181607047826822F4E0420A4328
:100B700082607047014600208968490700D501203E
:100B8000704710B50246002054680B0AC9B20C40E9
:100B90001168194202D0002C00D0012010BD01467E
:100BA00000208968090700D50120704738B5012168
:100BB0001C2003F0ABF9FF20ADF8000000248DF8F5
:100BC000034003258DF8025069460D4801F00CFBE7
:100BD0000120ADF800008DF803408DF80250694601
:100BE000084801F001FB2320ADF800008DF8034018
:100BF0008DF802506946044801F0F6FA38BD00004D
:100C000000080140000C014000100140002A426829
:100C1000C9B201D00A4300E08A4342607047000035
:100C200010B542680E4B0C791A400B6842EA042258
:100C30001343436083680B4A1340D1E902422243C5
:100C40004C7943EA44031A438260C26A097C22F465
:100C50007002491EC9B242EA0151C16210BD0000D2
:100C6000FFFEF0FFFDF7F1FF70B5072409290AD94F
:100C7000C568A1F10A0606EB4606B440A543B34099
:100C80001D43C56007E0056901EB4106B440A5437B
:100C9000B3401D430561836BC3F30154121B921CC7
:100CA00002EB82041F22A2409343A1400B438363C3
:100CB00070BD826B491E22F4401242EA01518163E9
:100CC000704770B5072409290AD9C568A1F10A0639
:100CD00006EB4606B440A543B3401D43C56007E09C
:100CE000056901EB4106B440A543B3401D430561CE
:100CF0001F23072A09D2446B521E02EB8202934043
:100D00009C4391400C43446370BD0D2A09D2046B8F
:100D1000D21F02EB820293409C4391400C43046338
:100D200070BDC46A0D3A02EB820293409C4391402D
:100D30000C43C46270BD816841F008018160704756
:100D40000029816802D041F4A00101E021F4A00152
:100D500081607047816841F0040181607047002123
:100D60000160017141718160C160012101747047AE
:100D700070B51E4C214694F83800B1F84250062850
:100D80001ED9B4F84A10B4F84C00A1EB000202F1ED
:100D90000902122A04D8FFF753FB0022144B0AE081
:100DA000884204D2FFF74CFB0022124B03E0FFF70E
:100DB00047FB0022104BFFF72CFAFFF786FB09E0F8
:100DC00005D12846FFF73CFB0C4A0D4BF3E70D49D4
:100DD00051F82000C5EB45116063B0EB410F03D91A
:100DE000C5EB45104000606370BD00004804002062
:100DF00000003440000033400000354067666666FE
:100E000066E64B400C8E000810B50C4C207840076D
:100E100013D5FFF7ADFF0A49A08E08800848303887
:100E2000018821F010010180001F018841F01001AC
:100E30000180207820F00400207010BD48040020BC
:100E400040040040F0B41448144B154A816804462D
:100E50001B782468526CCF0541F0080521F0080684
:100E60004FEA047413D5002C07DB090712D4002BBA
:100E700010D1142A0EDA856006E009070AD5002B86
:100E800008D1142A06DA8660F0BC05F0B5BD002C46
:100E9000F3DAEAE7F0BC7047A4020020FB0600206A
:100EA0004801002070B506464089204B204C4FF485
:100EB0008071002580B362887AB1012A0CD1E18863
:100EC000491C89B2E1803289914205D36580E58071
:100ED000FF2801D0401E708170BD7088228890422A
:100EE00001D9012200E00022184601F006FA7088BC
:100EF000B18801442088401C80B220808142EBD818
:100F00002580A088401C80B2A080F1888842E3D36D
:100F100001206080A58070BDFFE70022184601F027
:100F2000ECF9A580E58025806580F4E7000C0140A0
:100F3000B8050020FEE70000FCB505464FF6FF7639
:100F400000200C46ADF8006048F205078DF804005B
:100F500020E000BF15F8010B8DF8040001A9084638
:100F600002F0F5F8BDF800009DF8041080EA0120B9
:100F7000ADF800005FF00000BDF800100A0402D5D3
:100F800087EA410101E006EA4101401CADF800108A
:100F90000828F1DB641EDDD26946084602F0C1F87C
:100FA000BDF80000FCBD00000246002004E000BFC8
:100FB00012F8013B1844C0B2491EF9D27047000034
:100FC00070B5144A85B01088002413490194009428
:100FD000039420460494138807E00D8B009E35444B
:100FE0000095CD8B019E3544019515889D42F4D026
:100FF000401CC0B28028EED30098411107484180C0
:10100000848001984111064881830183818205B063
:1010100070BD000004070020A4020020D2050020BB
:10102000C004002030B50E4902880A800C4A43886B
:10103000083A13800B1F808818802024151F2C80ED
:101040000020401C80B27328FBD341F211100880AD
:1010500044F64800108047F2480018802C8030BDCC
:10106000202C0140114944F648000880091D46F62D
:1010700048000880091D41F2111008800B48001F2C
:10108000018841F02001018009480021A0F8641086
:10109000A0F86210A0F86010A0F85E10A0F85C1034
:1010A000A0F85A100348418181827047182C0140F2
:1010B000A40200206C000020F0B54D4B4D480021EB
:1010C000DA7A0778802A27F001057CD31C684A4B1E
:1010D00002F01F0253F82220484B14421A6802D033
:1010E00042F0200201E022F02002454C1A60454EF9
:1010F00094F800C0444CBCF1020FB4F904403FD155
:10110000B3F808C0CCF3C00ECCF3002CE64537D0C2
:101110003A4D2C3D95F802C0BCF1000F04D0BCF153
:10112000010F0FD0A9702FE05FEA025C2CD55FEAB7
:10113000826C29D44FF0010C85F802C027F0040519
:10114000057021E05FEA025C1ED45FEA826C1BD569
:101150005FEA477C11D447F004070770B0F802C07B
:10116000BCF1000F03D0418027F0010704E0448068
:10117000002C02DD47F0010707700227AF7003E083
:1011800005704180318041811C4DC78895F84650DB
:101190000FB9002C15DC077BAF4212D1B0F90270F9
:1011A00007F26667BC420CDC184FBF895FEA477CD8
:1011B00007D45FEA877C04D45FEA427C01D5FF074D
:1011C0000BD0077800E00FE05FEAC77C05D027F07E
:1011D00001070770418031804181C4800573500947
:1011E00060F3CB221A60F0BD057041804181F0BDF3
:1011F000D80500200C0900206C920008A4020020F1
:10120000FB0600201C010020D2050020140A00204B
:101210002DE9F04796B000240C940D940E940F9491
:1012200072B69048816941F400718161816941F42D
:10123000806181614FF4004002F03AFE8A4D002146
:101240002846FFF73FFB00212846FFF731FB874E7A
:1012500000213046FFF72CFB854F0021384600F077
:10126000BFF901204FF47041401C8842FCD328464E
:10127000FFF744FCB1463046FFF740FC384600F02B
:10128000BBF94FF46020CDE912048DF845400120F0
:101290004FF004088DF8440010948DF8508010A988
:1012A0002846FFF7BDFC01231A4605212846FFF713
:1012B00008FD0123022206212846FFF702FD012333
:1012C000032207212846FFF7FCFC012304220F21FB
:1012D0002846FFF7F6FC384600F08EF9684600F025
:1012E00036FA6148634E4C300090CDF80C80CDE961
:1012F00001648020CDE90440400006908000079002
:10130000202008904FF44050CDE909046946384642
:1013100000F000FA01212846FFF7D4FA01213846EF
:1013200000F05EF901212846FFF7C2FA47F230517A
:1013300015941598401C15908842FAD3012128462F
:10134000FFF7FEFCADF82C40A04640F2DC5A4FF40B
:10135000007420E05046CDF854801599491C159131
:101360008142FAD330880D9908440D9070880E9907
:1013700008440E90B0880F9908440F90F0880C999B
:1013800008440C9001212846FFF7DAFCBDF82C0038
:10139000401CADF82C00BDF82C00A042DAD30D980B
:1013A000354A40F3CF1633480A3006830E9941F38D
:1013B000CF1444830F9941F3CF1383830C9941F3E6
:1013C000CF1CA0F804C0ACF5C05C40F2C371ACF512
:1013D0009B7C8C450ED2A6F5C856363E8E4209D26D
:1013E000A4F5C854363C8C4204D2A3F5C853363B0E
:1013F0008B4203D3D18841F48041D180D188490404
:1014000007D41E49028B21F85C2F428B4A80808BC7
:10141000888000212846FFF755FA0021384600F061
:10142000DFF800212846FFF743FA00214C464846E2
:10143000FFF73EFA0220C102401C8842FCD3284636
:10144000FFF75CFB2046FFF759FB384600F0D4F865
:10145000FFF742FA0A493C20087062B616B0BDE8B0
:10146000F0870000001002400024014000280140E5
:10147000080002401E050020140A0020680C00200D
:10148000F8060020F0B53A4B3B4C93F85650394BD8
:10149000042D5B6C1DD0256840F22D465D1B6560F8
:1014A00043F6FB25B3F5FA5F33DDB3F5FA4F30DCD5
:1014B00041F6AD17A3F5FA535F4306EBA7364FF499
:1014C000B5777B4305EBA31375105B10C4E9065396
:1014D00021E043F6D017102641F26205BB4218DB2B
:1014E00044F25067BB420EDAA3F5645345F24C67F1
:1014F000D03B5F4306EBA736A66140F624767343E4
:1015000005EB232303E042F24713A3611B4BE36186
:1015100001E0C4E906654FF4BB73536044F24C2309
:10152000401AD3601060117C58430841116A01448D
:101530001162D069814200DD1062116A90698142B6
:1015400001DB084600E01062206211684FF4BB73B3
:101550005943137A194118410144B2F914008842E1
:1015600004DBB2F91200884200DC08B2F0BD0000D2
:101570006C000020480100202001002085EB0100C4
:1015800010B54FF40054204600F0ACF8002813D0FA
:101590000A49087840F008000870204600F014F866
:1015A0000021074800F01CF80648C17E012903D13C
:1015B0000021C1760121017710BD000072060020D4
:1015C000440002400C0B0020C10002D50249086013
:1015D000704702494860704704040240000002401E
:1015E0000029016802D041F0010102E04FF6FE72CD
:1015F000114001607047000001684FF6FE72114013
:1016000001600021016041608160C1603149314A5F
:101610000839904203D1486840F00F0006E02D4A97
:101620001432904204D1486840F0F000486070479E
:10163000284A2832904203D1486840F47060F5E7A8
:10164000244A3C32904203D1486840F47040EDE7B0
:10165000204A5032904203D1486840F47020E5E7B8
:101660001C4A6432904203D1486840F47000DDE7C0
:10167000184A7832904203D1486840F07060D5E74C
:10168000154A111F904203D1086840F00F0006E090
:10169000114A1432904204D1086840F0F00008600A
:1016A00070470D4A2832904203D1086840F47060B8
:1016B000F5E7094A3C32904203D1086840F4704093
:1016C000EDE7054A50329042EAD1086840F47020B4
:1016D000E5E700000800024008040240406880B2CC
:1016E0007047000001460020CA0001D5034A00E00F
:1016F000034A12680A4200D00120704700040240E9
:1017000000000240002A026801D00A4300E08A4338
:101710000260704730B5036847F6F07293430C6A75
:101720008A682243D1E904452C4322438C69224331
:10173000CC6922434C6A22438C6A22431A430260DA
:10174000CA6842600A6882604968C16030BD002191
:10175000016041608160C160016141618161C1617D
:10176000016241628162704710B5114C8CB000215A
:101770002046FFF735FF2046FFF73EFF0D4800905B
:101780000D480021CDE901016420CDE9030180204D
:10179000CDE905010791089109910A916946204612
:1017A000FFF7B8FF01212046FFF71AFF0CB010BD6C
:1017B00058000240043801409007002010B5012174
:1017C0008CB0084602F07EFB1E4C00212046FFF73D
:1017D00007FF2046FFF710FF1B4800901B480190B1
:1017E00000211020CDE902018020CDE904100691EE
:1017F0000791089109910A9169462046FFF78AFFEF
:10180000012202212046FFF77DFF01218DF82F10D4
:1018100004208DF82D008DF82E100E208DF82C0050
:101820000BA802F031F80F208DF82C000BA802F065
:101830002BF801212046FFF7D3FEFFF795FF0CB0F0
:1018400010BD000044000240043801402C07002075
:1018500030B540F6AA21204AC184838B1488E31A4C
:101860009BB20F2B10D312888283037E002253B1C8
:101870001A4BB3F90A30062B05DB194B1B78022BE8
:1018800003D0002B00D1828430BD164B40F68B254F
:101890005B6CA3F22D14AC420FD2428B521C92B25D
:1018A0004283642AF0D364224283B0F924208A421E
:1018B00001DA02EB2111818430BD41F29414A3427C
:1018C000FADBB0F92430002B02DDA3EB211100E09C
:1018D00000218184428330BD040700206C00002079
:1018E000FB0600204801002010B50446B0F90200B4
:1018F00043F6991148438113E06840F26662504311
:1019000001EBA030E060B4F9001043F699125143A6
:101910008A13216940F26663594302EBA1312161C8
:1019200004F0D0FC6061A18840F6AB22084440106E
:10193000A0F515415539E062914205D9A0F5F8515D
:10194000FF39521C91421DD249F25451884202DDA6
:10195000A0F5204002E0A0F5F850FF38206300EB2E
:10196000400040F34F002085B4F924104A429042D1
:1019700001DA104602E0884200DD0846E083228456
:1019800061848AE0A0F5FE42FF3A41F255518A4255
:1019900014D8A2F6AA20206300EB400040F34F00C9
:1019A0002085B4F924205142E183884201DA0846B7
:1019B00002E0904200DD1046404250E0A0F5D442E3
:1019C000AA3A8A4215D2A2F6AA20206300EB400070
:1019D00040F34F012185B4F924004242E283208480
:1019E000914201DA104602E0814200DC0846608440
:1019F00053E0A0F5AA42543A41F256539A4215D206
:101A0000A2F6AB20206300EB400040F34F0020859E
:101A1000B4F924104A42904201DA104602E08842AA
:101A200000DD08464042E083218419E0A0F58042B1
:101A300041F254539A4215D2A2F6AA20206300EB39
:101A4000400040F34F012185B4F92400E083424275
:101A5000914201DA104602E0814200DC084620840F
:101A600062841AE0A0F52852AB3A8A4215D2A2F657
:101A7000AA20206300EB400040F34F012185B4F918
:101A80002400E08342422284914201DA104602E0BF
:101A9000814200DC08464042A9E7B4F91E006FF419
:101AA000BF7148438013E080B4F92000484380139D
:101AB0002081B4F9220048438013608110BD704733
:101AC0001548164A4FF480410078042821D002F1CD
:101AD0003C03D08A9B88C01A00B22F2801DD001178
:101AE00008E0002801DD002007E00D4B984201DAF4
:101AF000184602E0402800DD40209389184400B2D7
:101B0000884203DC40F26661884200DA0846908130
:101B10007047918170470000FB060020C004002040
:101B2000C0FEFFFF38B54B484B4902880B889A1A14
:101B300092B20F2A71D30988484C01804FF0FF01FF
:101B4000E2884FF47A7355044FF4967002D516224A
:101B5000009103E0950403D515220091014670E041
:101B6000D50402D514220091F8E7150502D51322F9
:101B70000091F3E7550502D512220091EEE7950595
:101B800002D511220091E9E7D50502D51022009176
:101B9000E4E7150602D50F220091DFE7550602D5CE
:101BA0000E220091DAE7950602D50D220091D5E7C5
:101BB000D50602D50C220091D0E7150702D50B22DD
:101BC0000091CBE7550702D50A220091C6E7950799
:101BD00002D509220091C1E7D20702D00822009164
:101BE000BCE72289550702D507220091B6E7950781
:101BF00002D506220091B1E7D20702D0052200915A
:101C0000ACE7A27AD20702D004220091A6E7A2890B
:101C1000D40603D503220091A0E719E0140702D5EA
:101C2000022200919AE7540703D4940701D4D20703
:101C300002D00122009191E70020034602460146AE
:101C4000009002F02DFEBDE838400248FFF72AB9A7
:101C500038BD0000080A002004070020140A0020F4
:101C6000F0B55948594982880B889A1A92B29C2A31
:101C700064D30988818056490A880146002A0B7876
:101C800043F0020156D11646524A1C071568024617
:101C9000127822F0020274D54F4C0746E4887F7810
:101CA0005FEA845C02D547F0010701E027F00107F5
:101CB0004770A704477802D547F0020701E027F0F4
:101CC00002074770670401D4E70703D0477847F05D
:101CD00008074770640603D5447844F0040404E020
:101CE0001C0603D4447824F004044470EC0450D45B
:101CF000354C9A07247824F0100423D4324D4278CE
:101D00002F7A2D78012A45F0100514D0022A16D01A
:101D10002D4C042AA47804F1010C0CF0FF0C13D014
:101D2000072A25D0032A23D0052A21D0062A1FD02E
:101D300021F0100142E0B90702E00570F0BD39075B
:101D40000029FADB0470F0BDFA0601D41A060AD5A0
:101D50000170022C04D280F802C0BCF1020FF2D351
:101D600041F080012AE021F0100101708670F0BD81
:101D7000877A7F06F7D5032C04D8017080F802C05B
:101D8000F0BD0FE05107D8D51906D6D443F0800135
:101D900014E002704178CB0701D18907F0D522F019
:101DA00010010BE0E9040BD49907E9D4818AC82912
:101DB00002D2491C8182E3E743F00A010170DFE7A8
:101DC00002708682DCE70000DC06002004070020A9
:101DD00006070020A4020020140A0020094944F646
:101DE00048000880091D46F648000880091D41F694
:101DF000CC4008800348001F018841F02001018089
:101E000070470000182C0140084946F66800088019
:101E1000091D0880091D41F2555008800348001F24
:101E2000018841F02001018070470000182C01401A
:101E300010B5C28800210AB1032206E002890AB166
:101E4000022202E0428912B10122027000E0017018
:101E500004784FF4804344F6206244B1012C06D04C
:101E6000022C07D0032C01D14180818010BD43801A
:101E7000828010BD41F23331418040F6B731F4E742
:101E800030B5B1F86A5000231A240D22854202DCD5
:101E9000B1F9680030BD4D88854202DBB1F9000020
:101EA00030BD01EB82056D88854201DD144601E0FD
:101EB00013DA134604EB03024FEA52029A42F0D1BE
:101EC00001EB830231F8231054889288521A001BC8
:101ED000424301EB622000B230BD31F9220030BD37
:101EE000054920B1086940F0800008617047034847
:101EF000486003484860704700200240230167455E
:101F0000AB89EFCD06494FF47A70CA68D20705D085
:101F1000401E0004000CF8D1FF20704700207047DD
:101F20000020024012480321A0F1580280F8361028
:101F3000002191820F4A11860F4A1186D162D18306
:101F40001184518481620D498A6CB2F5206F01DBE6
:101F5000A3228262897A11B1816A49428162C16A8F
:101F600041F39101816288030549086270470000CE
:101F70006C000020A4020020280500204801002059
:101F8000700800200449002048810881C8628862E6
:101F900002490862704700006C000020940800208D
:101FA000F0B53B4988894A89801A80B20F2866D3E8
:101FB00088894881CA8937480B3A272A26D28A78E5
:101FC00022BB8268364B42F480728260324A354CC2
:101FD000354D12785607314A0AD4344E3688168069
:101FE000334A12881A80334A12882280324A09E022
:101FF000324E36881680324A12881A80314A128848
:102000002280314A12882A8001228A702F4B304D5B
:1020100019469A7F0968802A32D302F01F0255F8C8
:10202000222011422CD0826822F48012184E826045
:10203000123614461215B778521C62F38617254AD9
:10204000B77093F816C01778BCF1800F27F002061E
:1020500008D30CF01F0C55F82CC011EA0C0F01D15D
:1020600047F0020616701A7E802A0DD302F01F0276
:1020700055F82220114207D144F400218160F0BDBF
:10208000826842F48012D1E724F40021F6E70000D0
:10209000F8060020A402002048010020B804002017
:1020A000BA040020BC040020BE040020A8040020C4
:1020B000AA040020AC040020AE040020B0040020DC
:1020C000B2040020B4040020B6040020D80500208B
:1020D0006C920008C004002070B5204881890289F4
:1020E000891A89B20F292FD3818901811C4B1D4880
:1020F00019465D7A06681C4C096846F00402802D7A
:1021000007D305F01F0554F82550294201D126F0C8
:10211000040202609A7B802A17D302F01F0254F84F
:102120002220114211D1026822F002020260DA7A02
:10213000802A0ED302F01F0254F82220114208D147
:10214000016821F00801016070BD026842F00202DE
:10215000ECE7016841F00801F5E70000F80600200F
:10216000D8050020A40200206C920008F0B51D4C98
:102170001B4A4FF0010C94F83B5094F80AE01446C7
:1021800092F83C3094F838402B43651CEEB2154D64
:1021900095F83D700025BEF1FF0F0AD0BEF1000F8B
:1021A00006D18B4213D155700C2C01D282F83860C5
:1021B000F0BD834202D182F801C0F5E78B42F7D12E
:1021C0005570B80709E000BF82F83850F0BD83426F
:1021D000FCD1F84382F801C080070028F4D0F0BD9C
:1021E0004804002048010020F0B5CA78002502F01C
:1021F0000F03D20601D58A7813430A784FF00F0EE9
:1022000012F0FF0F4FF001021CD004680F8802FA91
:1022100005F63740B74211D14FEA850C0EFA0CF79C
:1022200024EA070703FA0CF43C43CF78282F02D0A6
:10223000482F02D002E0466100E006616D1C082DC7
:10224000E4D304600C88FF2C1ED944685FF00006BC
:1022500006F1080702FA07F50F882F40AF420FD1A9
:102260004FEA860C0EFA0CF7BC4303FA0CF73C431A
:10227000CF78282F00D14561CF78482F00D1056154
:10228000761C082EE4D34460F0BD0000F0B5144C79
:10229000002801DAE36900E06368420D120185B2AB
:1022A000C0F301579540C0F30346032F05D0C20287
:1022B0000AD50322B240934307E023F070626368BB
:1022C00023F07063636002E0AB4343F0706201B1DE
:1022D0002A43002801DAE261F0BD6260F0BD00002F
:1022E000000001400246002092680A4200D001200E
:1022F000704741617047016170470AB101617047E1
:10230000416170470F4A104B92F838105B5C834272
:1023100001D1012004E00D4B5B5C834203D100201E
:1023200082F83A0070470A4B5B5C834201D18120FE
:10233000F6E7084B595C814201D18020F0E7032089
:10234000EEE70000480100202C9600083E960008A9
:1023500032960008449600080A4810B501784FF0FC
:1023600000024C0708494FF0FF0389684FEA0171EA
:1023700005D5002901DA827210BD837210BD0029D3
:10238000FBDBF8E748010020A4020020F0B5194E5D
:10239000194C0022E31CA6F1060CB75CA518ED78D9
:1023A000FF5C0D430F43BD421FD01CF80270FF5C61
:1023B0000F43BD4219D015460023A618F6780E43E8
:1023C000C6545B1C1CF80220DBB2062BF5D3C17887
:1023D00081700179C17000214218491C15711CF8E7
:1023E0000550C9B20629F7D3F0BD521CD2B2032A58
:1023F000D3D3F0BDFE8D00084804002010B502467E
:102400000021064B06205C186478944200D10846EF
:10241000491CC9B20629F6D310BD000048010020AE
:10242000214810B590F8671000222048012936D1C4
:102430001F49898899BB1F491E4B4C6C40F6B83127
:10244000B3F86E308C4227DD1B49097821BB90F828
:102450002711491CC9B280F82711C8291CD380F85C
:1024600027210146D0F82C4191F82811A34203DD21
:10247000052908D2491C01E041B1491E80F8281104
:10248000C9B2052902D3012180F82611191B074C76
:102490002C3C6162C0F82C31B3F5FA6F03D280F89E
:1024A000262180F8282110BD680C0020A4020020FD
:1024B000D205002048010020FB0600204FF4C04256
:1024C0008260002141620E22828141F26202026139
:1024D000082282824FF46042C28201834FF0784228
:1024E000C0E9072140F6C41101807047B0F900101F
:1024F000B0F90220891A41600269037D4A431A41FA
:10250000436A13444362026A934200DD4262436AB3
:10251000C269934200DA42628268436A4A43017B9D
:102520000A410B41D118B0F918208A4201DA10464D
:102530007047B0F916008842FADC08B27047000014
:1025400010B514481449B0F88C200B889A1A92B22E
:10255000B2F5437F1DD90988A0F88C10B0F88A1015
:1025600020F8581F002242860C480D4CC2888280F9
:10257000C180C38983812489891AA4B2C4818160FE
:10258000E11A0161074A818AC182928A8282511AC4
:10259000816110BD4801002004070020300C00209C
:1025A000280500206C00002009480A49B0F8AA203C
:1025B0000B889A1A92B241F684639A4206D309882C
:1025C00020F8AA1F418881800021418070470000C7
:1025D00048010020040700200D480178C90702D0F7
:1025E0000C49098801E04FF6FA71C16509490120DB
:1025F0001039088007482438018841F00101018022
:1026000004481838018821F0180101807047000043
:1026100048010020240400400A49D1F8902012B15A
:10262000521EC1F8902031F88A2F521C21F81A2925
:102630004A6A521C4A628A8F521C8A8701F8380CF7
:1026400070470000480100201CB52D4890F83B3031
:1026500090F83C20934252D000248DF8044053401F
:102660008DF800309DF800300122012B08D09DF834
:102670000030022B09D09DF80030042B0AD00DE069
:102680001F498DF80420443108E01D498DF80420CD
:10269000463103E01A498DF8042048319DF80420A2
:1026A000012A2CD190F83D309DF80040154AA342F4
:1026B00017D090F83E309DF80040234208D0B0F883
:1026C0004C30A0F84A300B881488E31AA0F84C303C
:1026D00090F838302BB1B0F840301488E31AA0F8E5
:1026E000423012880A80A0F8402010F83E1F9DF862
:1026F0000020114300F801199DF8001001701CBD65
:10270000480400200407002070B5344D40212846BD
:10271000FFF7E8FD840080212846FFF7E3FD44EA47
:102720004004A9152846FFF7DDFD0443E1B22C4C17
:1027300094F870508D4250D04D4084F87010012DA7
:1027400003D0022D01D0042D47D194F87400A84382
:1027500084F8740094F87320AA420FD084F8735060
:1027600094F8722001238B401A4207D11A4384F84F
:10277000722094F87110491C84F8711094F871104B
:10278000042928D330B1012811D002280FD0042801
:102790000DD012E01348C18821F04001C18020789B
:1027A000002184F83B1020F06000207005E02178C3
:1027B00041F02001217084F83B000B4994F83B0064
:1027C00091F82720904204D081F827000749202063
:1027D000087000F00DF884F84C5070BD00100140F6
:1027E00048010020140A0020680C0020F806002090
:1027F00070B50D4D40212846FFF774FD84008021FF
:102800002846FFF76FFD44EA4004A9152846FFF764
:1028100069FD04430548072100F8704F017100214C
:1028200041708170C17070BD0010014048010020EE
:1028300070B5344890F83A10CA43920761D001F05D
:10284000030280F8392090F83D305B061B0E80F8BB
:102850003D30012A01D0812A02D15B1C80F83D3035
:102860000278D2074DD0DBB203F00102C3F340047B
:10287000A24246D1B0F84E400025641CA0F84E405C
:10288000204CA0F8505090F83E60A47AB24202D09A
:1028900080F83E200DE0A607B6EB837F02D080F8DB
:1028A0003F5006E090F83F30642B02D25B1C80F86A
:1028B0003F3090F84030642B0CD25B1CDBB280F8C8
:1028C0004030022B06D204F00103934202D10222CF
:1028D00080F84020012901D0002912D190F8382039
:1028E000C16D00EB820291610163D0E906121144CF
:1028F000D0E908231A441144826A1144C26A11447F
:10290000416370BD48010020FEE700002DE9F04F53
:1029100000BF00209E4E9F4AA6F51271A6F5BE7913
:10292000A6F1440B06F1440E804601F5E074A1F1D6
:10293000780301F5457A1D5C15F0C00706D0402FDD
:1029400051D0C02F77D0802F76D004E115F01F052D
:1029500004D0154440F080072F7201E082F808800F
:10296000012826D0022824D0032822D0042820D0F1
:1029700008281ED010281CD0874D55F820C0DCF840
:10298000005054F820703D40CCF80050824D55F86E
:1029900020C0DCF8005056F820703D43CCF80050C1
:1029A0001D5CAD0659F820502F6813D53AF810C0B9
:1029B0003EE051F820502F6854F820C007EA0C0779
:1029C0002F6051F820502F6856F820C047EA0C07B6
:1029D0002F60E5E7DFF8B8C10CF1F00C5CF820C01F
:1029E00007EA0C077EE015F01F0504D0154440F0FF
:1029F00080072F7201E082F8088001281DD002288C
:102A00001BD0032819D0042817D0082815D0102867
:102A100013D0614D55F820502F6854F820C007EAB4
:102A20000C072F605C4D55F820502F685BF820C0D4
:102A300047EA0C0756E00BE056E051F820502F68AB
:102A400054F820C007EA0C072F6051F82050ECE73B
:102A500015F01F0505D0154440F0800785F821705A
:102A600001E082F82180012825D0022823D0032804
:102A700021D004281FD008281DD010281BD0464D77
:102A800055F820C0DCF8005054F820703D40CCF8D8
:102A90000050414D55F820C0DCF800505EF8207021
:102AA0003D43CCF800501D5CAD0615D53A4D3AF8C3
:102AB0001070CC3514E051F820502F6854F820C025
:102AC00007EA0C072F6051F820502F685EF820C0ED
:102AD00047EA0C072F60E6E72D4D3AF81070E03D0D
:102AE00055F820502F6036E015F01F0505D015442D
:102AF00040F0800785F8217001E082F821800128EC
:102B000030D002282ED003282CD004282AD0082820
:102B100028D0102826D0204D55F820C0DCF80050D1
:102B200054F820703D40CCF800501B4D55F820C0A3
:102B3000DCF80050164F883757F820703D43CCF82A
:102B400000501D5CAD06B1D4114F3AF81050E03F73
:102B500057F820703D60401CC0B21128FFF4EBAE66
:102B6000BDE8F08F51F820502F6854F820C007EAD4
:102B70000C072F6051F820502F68DFF814C00CF1BB
:102B8000880C5CF820C047EA0C072F60D9E70000EA
:102B9000F8940008D8050020F49200084FF407715B
:102BA000C1824FF45861018340F61451818370470C
:102BB000F0B5C48AB0F900608681B0F90250C581D1
:102BC000B0F904300227002101220382AB4204DB6A
:102BD000B54202DDC78042810CE0B34204DBAE4265
:102BE00002DDC78041811CE09D4205DBB34203DD6D
:102BF000C2804781018115E0B54204DB9E4202DDBF
:102C0000C280418105E0AE4205DB9D4203DDC1800B
:102C10004281078106E09E4204DBAB4202DDC180B7
:102C200047810281C388458900EB430700EB4505D6
:102C3000BB89AE899B1B0FFA83FEA0F812E00689C0
:102C4000AB8900EB460CBCF80CC0A3EB0C038382F1
:102C5000B0F91830B7F90CC0A3EB0C0CB4EB4C0F67
:102C600004DA80F82010A3F1A10113E0A64503DDEA
:102C700080F82010B9890BE026B1012E04D0022E75
:102C800010D004E0062100E0052180F82010A98979
:102C9000091B6D31418309B2B1F5586F04DB5B1E2E
:102CA000438304E00421F0E7002900DC4283418BE8
:102CB0008183F0BD0B49002288760A62CA614A62AC
:102CC000094A32F9103002EB40028B62B2F902205D
:102CD000CA62064A32F810000882A1F86000A1F822
:102CE00062007047F8010020569600084A960008D6
:102CF0002DE9F05FF848F94982880B889A1A92B258
:102D00000F2A44D309888180F54982460127088823
:102D1000F44CF54E002578B3401E0880E573F34966
:102D2000A5622068B1F90210430742F6AA2218D41E
:102D3000F38843F40053F380EC4B1B789B0709D5D1
:102D4000A36823F08003A360A4F87C5084F87E502D
:102D500084F87F50C30404D484F8F070C4F8EC50B5
:102D600003E084F8F050430707D4914205DB84F870
:102D7000F470A4F8F25004E010E084F8F450430733
:102D800003D4914201DBC00703D084F81151BDE8A0
:102D9000F09F84F81171A4F81251F8E7B4F8180103
:102DA00043F69821884202D2401CA4F8180101F091
:102DB0008DFDDFF83C83DFF820B398F85000ABF1CD
:102DC000180B10B1FEF778F905E09BF8001021F020
:102DD00001018BF8001098F8630010B1FEF732F88B
:102DE00008E0A068C10502D520F0080001E040F02D
:102DF0000800A060FFF714FB00F0C0F9BD4841F2E5
:102E00006801436C4FF400608B4201DBBA4904E077
:102E1000B3F57A6F02DAB849091D086098F85100D5
:102E2000C646C107DFF8BC82B448DFF8D492A8F1E7
:102E30002C0839D0817B802932D3217889072FD47F
:102E4000E17B88F80510A949424691F800C02CF0B2
:102E5000020C81F800C0ABF80250CBF814509BF87C
:102E600000C02CF0010C8BF800C0B179490612D4D7
:102E7000518941F2883C614503D2491CA8F80A10E7
:102E800012E040F63C70834201DD0020F9E00420AE
:102E900088F80370F5E0D5700020A8F80A50F0E03B
:102EA00088F80350A8F80A50A1680A0501D508203F
:102EB000E7E09EF83FE05FEACE7240D0E27B88F820
:102EC0000520437A802B5BD323785B0730D4F388CB
:102ED0009B0403D521F02000A06030E0ABF8025045
:102EE000CBF814509BF800C041F020012CF0010CED
:102EF0008BF800C0A160C17D802909D301F07F0358
:102F000000684FF00041D940084201D1277100E02C
:102F100025712079C00702D15FEA8E7005D50320A4
:102F2000032A01D088F80870ABE00020A562A8E071
:102F300021F02000A060F08820F40050F08094F888
:102F40002601012821D094F846104FF48047F1B1B2
:102F500043F23332012932D0032999F8001069482D
:102F600043F69913C1F381012CD0012941D00229E4
:102F70003FD090F85600042838D0A4F814713EE0F1
:102F8000206840F004002060A4E7092079E099F867
:102F9000000042F6CC41C0F38100012809D002288C
:102FA0000AD042F6B86000BFA4F81401A4F8441097
:102FB00027E0A4F81411F9E742F26660F4E7A4F8F8
:102FC00014211CE001290AD0022908D090F85600EB
:102FD00004280BD0A4F81431A4F8447011E0A4F82C
:102FE000147190F85600042814D0F5E7A4F8147171
:102FF00010E0A4F8147190F8560004280AD0A4F840
:103000004420FEF759F89BF80010C90705D0BBF81B
:10301000021004E0A4F84430F3E734488188AAF8A9
:10302000121008B2B4F944104843C0F38F3140463F
:10303000A8F81210B94200D9478233490978C90665
:1030400005D5428A41F233318A4200D24182218938
:10305000C1F3C002C1F300218A4205D1428A40F681
:10306000CC418A4200D94182B17AC90700D0458259
:10307000B8F81200A06200287FF707AF2348057058
:1030800002209AF81A1099B9022841D080B1194942
:103090000B789D0608D5B5796D0605D51A4D2D78A6
:1030A000ED0965F386130B70F18821F40A61F18054
:1030B0001049496C4E290ADBF1880B0607D521F02F
:1030C0008001F18009490B7823F002030B708AF824
:1030D0001A00E0735BE600002409002004070020CA
:1030E00006070020A4020020140A0020D2050020B8
:1030F000680C002048010020100C0140D805002079
:10310000C00400206C000020DC060020180700200E
:10311000B9F83830002BBAD143F69823A9F83830E3
:10312000B5E770B500230C8863F30F02012505FA9B
:1031300003F6344206D0C3F10F0605FA06F1114337
:1031400061F30F025B1C102BF1DB028070BD70B5C8
:1031500000230C7863F30702012505FA03F63442D5
:1031600006D0C3F1070605FA06F1114361F3070221
:103170005B1C082BF1DB027070BD0000F0B51F482E
:1031800090F866301E48012B816821F4006232D12C
:103190001C4BDE8874062ED41B4D0F054FF0000427
:1031A000B5F902501ED4194A526C642A11DC40F65B
:1031B000386295420DDAB2040BD4027852070ED46D
:1031C000B0F8D42040F6B835AA4203D2521CA0F879
:1031D000D420F0BD41F4006181605C81F0BDA0F8B5
:1031E000D440F0BD41F2CD018D42FADD997AC90794
:1031F000F7D18260F3E78260F0BD0000680C002028
:10320000A4020020140A0020D2050020480100205A
:10321000F0B5364D364F044695F83B0097F83B1015
:1032200023780843EE1C6278834205D1E07811468A
:10323000FEF79CFF207908E094F802C084450CD189
:10324000E1781046FEF792FFE07905F82F0F287815
:10325000805D6870287BE877F0BD82421DD16146B1
:103260001846FEF783FF95F84E1095F83B00814213
:1032700007D1B97A09B1A17900E0617985F82F10F9
:103280001EE06978012901D0A17922E0617927E067
:10329000297841F00401297012E0E1788142DBD104
:1032A00019466046FEF762FF95F84E1095F83B0010
:1032B00081420AD1B97A09B1617ADFE7217ADDE783
:1032C00015F82F1F895D6970C5E76978012906D057
:1032D000617A85F82F10B97A0029F1D1D8E7217ADF
:1032E00085F82F10B97A0029EAD0D1E748040020E8
:1032F000480100200B48017821F0020100F8381B3A
:10330000002100F8181941778177332181854185A3
:1033100008214184012100F81F1C034880F839105E
:103320007047000048040020480100200D4900B506
:103330000B4851F8012F40F8032F898881800848F5
:1033400001210930FFF722F8054802211330FFF769
:103350001DF8034804211D305DF804EBFFF716B893
:103360004804002048010020094944F6480008802C
:10337000091D46F648000880091D41F21110088019
:103380000348001F018841F02001018070470000C0
:10339000182C01402DE9F047664C674B0025A078BA
:1033A0000126654A103305287ED2DFE800F00313BA
:1033B000113E1100108820F0010010801D805F4830
:1033C0000580001F0580001F0580FFF7CDFFA67058
:1033D000BDE8F087594941F244401C3908805749FB
:1033E00045F6580024390880091D47F25800088026
:1033F00052492020283908800020401CC0B2732880
:10340000FBD3FFF7B1FF4C4984F85C502C3147F6F1
:10341000906008804848143006801D80108840F075
:10342000010010800220A070D2E700215FF00100AF
:1034300004EB410204EB4003B2F85020B3F85030E3
:103440009A4200D20146401CC0B20628F0D33C4844
:10345000405C84F83900FFF74DFF1D2000F0F3F9C0
:1034600000F076F8374E38484FF4807996F83B10E4
:10347000012904D002291BD0042930D047E0402183
:103480008046FEF72FFF870080214046FEF72AFF87
:1034900047EA400749464046FEF724FF074347F006
:1034A000010084F83B0000E03DE0224809302CE0B8
:1034B00040218046FEF716FF870080214046FEF738
:1034C00011FF47EA400749464046FEF70BFF074316
:1034D00047F0020084F83B001648133015E0402105
:1034E0008046FEF7FFFE870080214046FEF7FAFE89
:1034F00047EA400749464046FEF7F4FE074347F0D7
:10350000040084F83B000B481D3002F0B5FD94F830
:103510002F0086F838001D2000F0ABF90420A070C1
:103520000A48057054E7108820F0010010801D80C3
:10353000A5704DE748040020000800403C2C0140E5
:10354000048E00084801002000100140FB06002006
:103550002DE9F041344C14F82F0F344DE072402126
:103560002846FEF7BFFE860080212846FEF7BAFEF9
:1035700046EA4006AF1539462846FEF7B3FE064335
:10358000207BF1B22F3C814215D084F83C004021D1
:103590002846FEF7A7FE860080212846FEF7A2FEF9
:1035A00046EA400639462846FEF79CFE064384F864
:1035B0003B60FFF749F81E4D95F83B00012827D0E6
:1035C000022828D0042829D0174894F83B10273027
:1035D000085C04F8300F14F80109FEF70FFF04F837
:1035E0002F09A87A00B10120607001F0FBF994F86E
:1035F0004E0094F83B10884206D094F83800062814
:1036000002D2401C84F8380084F84E10BDE8F081E6
:103610000548093004E00448133001E002481D3039
:10362000BDE8F041FFF7F4BD480400200010014060
:10363000480100202DE9F041524991F87200AA2872
:103640007ED191F8730055287AD14F4C00200A5C46
:103650002254401CC0B27428F9D34C4E2069C6F8DD
:103660000100A08AA6F80500D4F81600F060D4F88E
:103670001A003061D4F81E001234706102F0A2FC0E
:103680004349608A888102F0B7FC207D123CC00764
:10369000307802D040F0040001E020F004003D4901
:1036A00030704FF480403C4D886114F8280F85F845
:1036B0002000608B6880A08BA880E08BE880208C45
:1036C0002881608C354F688194F8240087F8D200F7
:1036D00014F8011C304686F83B100026C0F89460B0
:1036E000FFF724FE2E48A18E0183E18E4183218FB6
:1036F000818394F84210283C012908D0022901D086
:10370000032909D0297821F00C01083107E0297834
:1037100021F00C01091D02E0297841F00C0129700B
:1037200094F86E20012162B1012A01D0022A0BD047
:1037300087F8461094F864301A4A4BB1518108E07A
:1037400014E087F84660F5E7022287F84620F1E7A3
:10375000568194F8701001290AD094F86D1051B177
:1037600001290BD04FF48051A0F87610BDE8F0810C
:1037700044F21C71F8E74FF40051F5E741F255515E
:10378000F2E7000000FC0008680C0020480100205F
:103790006C000020000C0020C0040020A4020020C7
:1037A00028050020140A00207CB50121082000F023
:1037B000ADFB4FF48070ADF8040010248DF8074085
:1037C00001208DF8060001A91548FEF70DFD012125
:1037D000092000F09BFB01211248FEF757FD08204D
:1037E000ADF8000004208DF803000F4E03258DF87E
:1037F000025069463046FEF7F7FC08213046FEF7D6
:1038000078FDADF800408DF803408DF80250694610
:103810003046FEF7E9FC10213046FEF76AFD7CBD1C
:103820000014014000023000000C0140FEE7704728
:1038300000F01F02012191404009800000F1E020CA
:10384000C0F88011704700F01F020121914040092B
:10385000800000F1E020C0F88011704700F01F02E6
:10386000012191404009800000F1E020C0F80011E2
:10387000704700F01F02012191404009800000F1D3
:10388000E020C0F80011704770B50F23C4780178AC
:103890000122F4B1144C2468457804F4E064C4F5C2
:1038A000E064240AC4F10406E3408478B5401C4077
:1038B0002C4301F1E021230181F80034007800F06D
:1038C0001F018A404009800000F1E020C0F800217B
:1038D00070BD01F01F0082404809800000F1E02027
:1038E000C0F8802170BD00000CED00E002490843E3
:1038F00002490860704700000000FA050CED00E086
:103900002DE9F05F00261D20FFF792FF6C4CDFF8D9
:10391000B4B1A4F1B000A77E90F83810DFF8A8E1A8
:10392000DFF8A8A100258F427ED0E776A176626AF3
:10393000036B5A434FEA12499BF80820120702D53D
:103940001EF8012000E00A4694F812C0BCF1010FF5
:1039500009D004EB4206B6F902C0C4F828C0B6F993
:103960000460E6620CE043F6FF7CC4E90A5C90F870
:103970003DC05FEACC7C01D012B102E0052A00D143
:10398000012600EB47074FF0804CBF893F04B7FB8F
:10399000F3F3E361476BBCFBF7F7276294F813C0BE
:1039A000BCF1000F06D0BCF1010F05D03B4403EB86
:1039B000D3735B10636201E03B466762DFF810C1BE
:1039C0004FF6FF7707EA8307ACF808709AF80070A3
:1039D00090F80A8090F83DC0082F08F003070CF01B
:1039E000030C05D067450BD1B8F1000F05D008E0F6
:1039F000674505D0B8F1000F03D05B42636200E079
:103A00006562C6B1636A002B03D006DD228D05E036
:103A10000AE0304B33F8122000E0A28DA4F86020B9
:103A2000227822F0200222709AF80020042A07D07F
:103A3000082A05D012E0B4F8603003EB0902EDE784
:103A400080F8405065629BF80800000701D51EF819
:103A50000110204830F81100A4F860001E49606A87
:103A600009883E314843B4F8601001EB204006B2AB
:103A70001D20FFF7F3FE606A002807D021784FEA87
:103A800081600ADD002804DAA08D09E0B4F8600046
:103A900006E0E06AB04208DB0CE0002802DA208D84
:103AA000208208E0A06AB04204DD208241F02000BC
:103AB000207000E02682257565752586BDE8F09F9B
:103AC000F8010020A402002038960008FB06002020
:103AD000EC0900204A9600082404004043184FF4E3
:103AE0008042934210DD904202DD104600210BE03F
:103AF000914202DD0020114606E08003B0FBF3F0A6
:103B000000B2C0F5804109B241EA004070470000B0
:103B10002DE9F04300234FF4BB740E25446003628B
:103B2000058144F24C260827C6600782DFF83490EE
:103B300043F6FF7CA0F81290A0F814C04FF0704834
:103B40004FEA8C32C0E906824C600B620D81CE6078
:103B50000F82A1F81290A1F814C0C1E90682BDE855
:103B6000F083000000C0FFFF00214162094981602D
:103B70000E2181814FF6BF510161082181824FF4EE
:103B80004041C18243F6FF7101830907C1610249C7
:103B900001627047638A010000C0FF0F064941F6C9
:103BA000A260088005480168054A01F4E0611143FC
:103BB0000160BFF34F8FFEE7442C01400CED00E0A5
:103BC0000400FA0538B501210D2000F09FF94FF4EB
:103BD000E060ADF8000018248DF8034003258DF84F
:103BE000025069460D48FEF7FFFA4FF46040ADF809
:103BF00000008DF803400A4C8DF8025069462046BB
:103C0000FEF7F2FAA014ADF8000048208DF803008A
:103C100069462046FEF7E8FA38BD0000000801407A
:103C2000000C0140F0B50121CE028DB0304600F00D
:103C30006DF95A4F384601F047FB08A801F070FDB6
:103C40004FF45860ADF824000024ADF82040202047
:103C5000ADF82200ADF8264008A9384601F012FD63
:103C60000021384601F065FD4FF6FF71384601F03E
:103C70006AFD01220021384601F0F6FC0121384698
:103C800001F0DEFA04A801F0F6FAADF81060701049
:103C9000ADF81200ADF81440A220ADF81600700087
:103CA000ADF81800ADF81A40ADF81C4004A938462C
:103CB00001F0D0FA6020ADF80000ADF80440ADF896
:103CC0000840ADF80C40ADF80240ADF80640ADF844
:103CD0000A40ADF80E406946384601F0B5FB69462A
:103CE000384601F0F7FB6946384601F03DFC70208C
:103CF000ADF800000125ADF8045040F61450ADF8C1
:103D00000600ADF80840ADF80C40ADF80250ADF833
:103D10000A40ADF80E406946384601F069FC0121C1
:103D2000384601F0B1FA0821384601F0CDFB3146A2
:103D3000384601F00FFC0821384601F053FC3146AB
:103D4000384601F087FC7021384601F090FC1820BD
:103D50008DF82C008DF82D408DF82E408DF82F50C9
:103D60000BA8FFF791FD0D480C30018841F0800150
:103D700001800A481430018841F001010180001FD0
:103D800004800121384601F089FA8DF8285001217C
:103D9000384601F08DFA0DB0F0BD0000002C014056
:103DA0007047000070B50189C1EB411101EB410181
:103DB000CA0B42810B49104603F0ECFC09480C3851
:103DC000B0F90C200168B0F90E4001FB02F5436820
:103DD000614303FB145503FB0211AD138913C0E9C2
:103DE000055170BDF809002040F2134141600821DF
:103DF00081608621C1604FF4804101614942416187
:103E000000210162C16270470162704710B50188EC
:103E10004288891A09B20183B1F5005F02DBA1F57E
:103E2000804104E011F5005F02DC01F5804101836F
:103E3000B0F9182041685143C1618368846A5343D3
:103E4000C2681B12624303EB2222036A1A44114424
:103E500002628A13426241698A4203DB01698A4233
:103E600000DC11468A1AC0E90A21028E4FF403735E
:103E7000594302EBA13202860B4A1278082A04D178
:103E80000A4AD36E03EBA131D166B0F93010B1F517
:103E9000804F02DDA1F5804103E0002902DA01F53F
:103EA0008041018610BD0000FB060020280A00208A
:103EB000034A516821F440410143516070470000BA
:103EC00000100240044A0029516901D0014300E07A
:103ED000814351617047000000100240044A0029EC
:103EE000D16901D0014300E08143D16170470000F6
:103EF00000100240044A0029116901D0014300E08A
:103F0000814311617047000000100240044A0029FB
:103F1000916901D0014300E0814391617047000045
:103F200000100240044A0029D16801D0014300E09A
:103F30008143D160704700000010024030B5244931
:103F40004A6812F00C03234A03D0042B01D0082B3B
:103F500026D002604A680F231F4C03EA1212A35CAA
:103F60000268DA4042604B68072505EA1323E35CE8
:103F700022FA03F383604B6805EAD323E35CDA405B
:103F8000C2604B68032403F4404104EA933303EB1B
:103F90009161114B1B1F595CB2FBF1F1016130BD06
:103FA0004A680E4B1A404B68140103F4803303D562
:103FB000C2F38342113202E0022404EB924213B1B5
:103FC0004B689B0301D5064B00E0024B5A43C0E708
:103FD0000010024000127A000400002000003C089B
:103FE00000093D002DE9F041274CA615402120464F
:103FF000FEF778F9850080212046FEF773F945EA3F
:10400000400531462046FEF76DF90543EDB24021EB
:104010002046FEF767F9870080212046FEF762F907
:1040200047EA400731462046FEF75CF90743F8B2FD
:10403000A842DBD140212046FEF754F987008021B9
:104040002046FEF74FF947EA400731462046FEF783
:1040500049F90743F8B2A842C8D140212046FEF7EB
:1040600041F9870080212046FEF73CF947EA4007E6
:1040700031462046FEF736F90743F8B2A842B5D1DB
:104080002846BDE8F08100000010014010B502682C
:10409000416802FB02F301FB01330D4CA34211D92D
:1040A0001B0E0F3B0B4C9BB212B234F8133009B20B
:1040B0005A43594342F38F3241F38F31C0E9022111
:1040C000012102E0C0E902210021017410BD0000BD
:1040D00040A45D0F148A00082DE9F05FFE48FF49F7
:1040E00002880B889A1A92B20F2A76D30988018027
:1040F000FB4802468189D2884B0703D48B0701D441
:10410000CB0702D042F4007201E022F40072C280B8
:104110008146080702D44846C90604D5B9F80610F6
:1041200041F0010102E0C18821F00101A9F8061067
:10413000EB48FDF77DFEEB484FF4804AB0F93A10AA
:10414000514502DA491C418701E0A0F83AA0E64E49
:1041500041F6CC41E54DB06C884203DDA86820F003
:104160001000A860E24AE34FE3481188002411B12F
:10417000491E118008E0E98F41B1491EE987DF49F6
:104180000A7822F002020A70EC732DE0B9F80610EA
:104190004B0419D4B9F80C20D30615D4120713D444
:1041A0000A0611D48A060FD40A050DD44A0603D58F
:1041B000D34A1278120607D54A0705D4CA0503D494
:1041C0000A0701D4C90609D5CE49EC73CE4A3C7022
:1041D000CC83148081F82A4007E07AE039780129FD
:1041E00003D10178062900D13C703978DFF8FCB2A0
:1041F0004FF00108ABF12C0B0A2978D2DFE801F06F
:10420000FE690569FDFC6977CCE3E87B09281AD0D3
:10421000DFF8F89202286CD0B5F8400010B399F896
:10422000680040F63A22012822D0C5F8D84085F827
:10423000EA40CBF82040B5F9301001F21D50904211
:1042400026D8102325E0A4484430FEF737F9FDF7BF
:1042500069FE716CCBF8281041F27C510920CBF833
:1042600018108BE1AA48018B2986A5F8408015E03B
:10427000A848C5F8D80085F8EA80B5F9301001F2F1
:104280001D53934201D8102300E02023102202E0A6
:1042900020231022002000F00FFB288699F86830B8
:1042A0009D49012B736C40F2DC504FF4927212D096
:1042B000834204DA9648B0F90A00904212DBB5F85E
:1042C000402040F6C410521C92B2A5F84020824211
:1042D00008D2BDE8F09F8342FBDA8D48B0F90A00AE
:1042E0009042F6DA3C7085F8EA404C83F1E7B6E09C
:1042F000FFE7716CCBF828108BF807808748A5F88A
:10430000404085F8EA40427F5E4652B1C17F91B39A
:10431000C4774477B5F93000504539DDA5F830A0B1
:10432000D7E708B27E4901F013FCA5F8E400A96ABA
:10433000814200DA084600B2B08299F84D10002997
:10434000B5F9301002D03623052201E0A3230A225A
:1043500000F0B2FA2886B5F91601B5F914118842B1
:104360000ADA317901F10101C9B231710429D1D3DD
:104370003471401C02E007E003DD801EA5F8160141
:10438000C8E7A5F81611C5E740F266602886C1E7C0
:1043900000289EDA2C869CE76249D5F8DC0088422A
:1043A00002D2401CC5F8DC00E87B082803D1D5F810
:1043B000DC00884203D33C70C5F8DC4089E7BDE8E7
:1043C000F05F02F02DBCE87B092801D02C8645E186
:1043D000DBF81C005F46401CCBF81C00022809DDFE
:1043E000388D012301B2388B052200B200F064FA47
:1043F000FC61B862398D02E00FE00AE012E0364855
:1044000044300180B6F844104180FEF76FF82886EA
:104410005FE7BDE8F05F04F0BFB9434800780928C2
:1044200058D056E7414ADFF808E11188491C8BB2A1
:1044300040491380C82B04D391F800C0BCF1010F90
:1044400019D0B3F5FA7F04D391F800C0BCF1020F84
:1044500011D0B3F57A7F02D30B78032B0BD0E97B15
:10446000891E082937D2DFE801F011BEFBF70536B7
:104470009A04E8E62DE70C701480B9F8062022F4BF
:104480000062A9F806208EF80080E8E7FDF764FFD7
:104490003078400611D52848807804280DD0706CFB
:1044A00082280ADAB07A96F83D1000F0030001F095
:1044B0000301884201D001F04BFD38780628A7D0CF
:1044C00086F83F40B06C40F311011148C162890386
:1044D0001A4835E0C2E0DFE024090020040700208C
:1044E000140A00202805002048010020A402002012
:1044F00008070020FB060020FC060020D205002053
:10450000DC060020B808002028000020680C0020ED
:104510006C0000209AF9FFFF94090020300C002065
:10452000488D0008C0D4010060020020180000205F
:1045300014000020150000204804002094080020EA
:104540000162FDF7EFFC8BF80780B5F81401A5F8C0
:104550001601706CA5F88240B0F5437FA5F880A0E5
:104560000EDDA86840F48060A86096F83810052930
:104570007FF4BCAE40F01000A8606BE03870A8E695
:10458000A96821F48061A96040F28A21884204DA96
:104590003078400601D402F02FFAA868EAE7716C7F
:1045A000B1F5437F04DA0178062901D004706BE08D
:1045B0003D48017821F040010170FDF7B3FCA5F8FA
:1045C00016A1FDF7C9FE394810F8281F21F0010196
:1045D00001703749C5F8DC400C6236490C6208218D
:1045E0003970446475E699F80600C006C7D4706C4B
:1045F000B0F57A7F32DDFDF7AFFE3078400611D599
:104600002D48807804280DD0706C82280ADAB07AA0
:1046100096F83D1000F0030001F00301884201D03C
:1046200001F096FC86F83F40B6F84800288601B2B3
:104630002C46514501DDA4F830A0FDF773FCA068BD
:1046400040F48060A06096F83810052997D140F0BA
:104650001000A060022091E713E001E03C7038E612
:10466000716CB1F5437F02DA017806299ED1B9F861
:10467000061021F02001A9F80610FDF76DFE0420B8
:104680007CE70078062802D087F8008021E60B49F5
:1046900009200870052071E707498C7004700848EC
:1046A00080F8564076E600000A070020280A00201D
:1046B00070080020940800204804002060020020B8
:1046C0006C00002030B585B001210420FFF71EFCEE
:1046D0004FF40040ADF8100048208DF8130004A9F5
:1046E0001848FDF781FD01210846FFF7F7FB40F66A
:1046F0008C20ADF8040003240020ADF80040ADF894
:104700000200ADF806004FF080456946284600F0EB
:10471000B9FF1C208DF80C008DF80D408DF80E406F
:1047200001208DF80F0003A8FFF7AEF80122114613
:10473000284600F081FE0121284600F0AFFD05B0BB
:1047400030BD000000080140704700002DE9F04135
:10475000304CE07800285AD12078002857D0401EED
:1047600010F0FF00207052D14FF49670208272B684
:10477000294F45F2AA50A7F872000020FDF7B0FBC0
:10478000264D13202860FDF7BDFBA8BB3420E86050
:1047900002202861224E6E61286940F040002861A5
:1047A000FDF7B0FB40BB00211E4A08465FEA2553D7
:1047B00012F800C0BCF1FF0F00D00121401C80B2F4
:1047C0009842F5D3C1B9C4E9067639260127A06914
:1047D00010F8011B10F8012BA061E06901EB022128
:1047E00002886A612F6120F8021BE061FDF78AFBF5
:1047F00010B9761EB6B2EAD20120FDF771FB62B69F
:1048000001F0FAFB0848816821F480418160BDE82D
:10481000F0810000F8060020680C00200020024013
:1048200000FC000800FC0008A402002019480168F0
:1048300041F010010160016821F00301016001688D
:1048400041F00201016014484168416041684160E3
:10485000416841F480614160416821F47C1141600C
:1048600041680E4A11434160016841F08071016066
:1048700001688901FCD5416821F00301416041686C
:1048800041F0020141604168C1F381010229FAD17E
:10489000704700000020024000100240000028087D
:1048A00030B5044C039D6080A180E2802381658146
:1048B00030BD0000080A00200A44824201DA10B22A
:1048C0007047C91A8142FBDD08B27047F0B53E4817
:1048D000DFF8F8E03E4CC17F467A056800233D4A88
:1048E0003D484FF0010C802925D301F01F015EF8EF
:1048F00021100D420146096802D041F4805101E0C7
:1049000021F480510160CF0411D48F040FD5977A20
:10491000FF0705D05381277827F00207277006E0AC
:1049200090F846709FB1012F14D080F846300F0BDD
:1049300067F34D310160802E25D306F01F015EF82C
:1049400021100D42016809D041F0040108E080F80F
:1049500046C0ECE7022780F84670E8E721F0040142
:1049600001604D070BD44D0509D5957AED0706D0AA
:104970005381257825F002052570C0F898308C0801
:1049800064F38A210160917AC90718D1134991F81B
:104990006410012913D11249496C32290DDC0178C8
:1049A00049070AD50189090507D4D0F8981047F2BC
:1049B0003054A14204D9A2F80AC0C0F89830F0BD22
:1049C000491CC0F89810F0BDD80500206C92000872
:1049D000D2050020140A0020A4020020680C002048
:1049E0004801002010B5FCF7C3F90F48018821F0F9
:1049F000020101800C49183109880C4A928E114439
:104A0000094A3432118008490C390A8842F00102FF
:104A10000A80011D0A884FF6ED531A400A8001886A
:104A200041F01201018010BD0C0400404804002038
:104A300006480188491C89B20180B1F57A7F04D308
:104A40004188491C41800021018070471C070020DB
:104A50000F4810B5016841F00101016041680D4A3D
:104A60001140416001680C4A11400160016821F465
:104A700080210160416821F4FE0141604FF41F0173
:104A80008160FFF7D3FE05494FF00060086010BD5C
:104A9000001002400000FFF8FFFFF6FE08ED00E006
:104AA0002DE9F0412F4D28884FF00004000629D54C
:104AB000FCF7D8FA2C4A2D4807231778C8262C492A
:104AC000012F22D02B4FB7F806C0BCF1000F3ED00B
:104AD000B0F80CC04CF0080CA0F80CC0B0F806C040
:104AE0002CF4006CA0F806C0886820F004008860F0
:104AF000FC801370CE8700204FF49661401C80B27A
:104B00008842FBD32C80BDE8F0811B4F97F800C092
:104B1000BCF1010F0FD0BCF1020F11D0B0F806C0EC
:104B20004CF4006CA0F806C0886840F0040088606F
:104B300005203870DDE7B0F80CC04CF0080C03E03D
:104B4000B0F80CC04CF0100CA0F80CC0F0E70B4F04
:104B50003C70C78847F40067C780886840F004004D
:104B60008860C6E7102C0140FB060020140A0020D4
:104B7000A402002024090020FC06002019070020C0
:104B8000704700002DE9F0434FF08040018A21F08A
:104B900001010182AC48007800287CD1AB4FF87B42
:104BA000002878D1AA48406C322874DCA948806873
:104BB000DFF8A4924104A94DB9F804004FF00004B5
:104BC00003D4401CA9F8040028E1002874D02978F7
:104BD000012611B1012912D017E14946B0F5BE7F77
:104BE000FAD92E70CC718C71EC702C72287A0A185C
:104BF000401CC0B2147228720F28F7D305E1B9F82F
:104C000002204946824201D9EE7100E0EC719248DF
:104C10008A7908300F2A15D2CB79082B0BD2C3F131
:104C20000708EB7912F800C003FA08F36344135441
:104C3000CA79521CCA71CA79082A03D18A79521CCE
:104C40008A71CC7199F80610C8460F2973D10D21CD
:104C5000FCF772F9A881010A6970C0B2A87088F8DF
:104C6000064098F816208A4265D198F815108142BE
:104C700061D198F80BC07A49032302227948BCF12C
:104C8000000F10D0BCF1010F02D0BCF1020F14D004
:104C900080F86A2000E0CBE091F800C02CF00C0C0A
:104CA0000CF1080C0FE080F86A6091F800C02CF05D
:104CB0000C0C0CF1040C06E0A9E080F86A3091F8C5
:104CC00000C04CF00C0C81F800C098F80C10B6EB4A
:104CD000111F04D180F86E4087F846400EE0B2EB19
:104CE000111F04D180F86E6087F8466006E0B3EBD0
:104CF000111F03D180F86E2087F846200B0717D0CC
:104D000001F00F01012901D0022915D080F86C6053
:104D10002C7198F80D102A7906FA02F30B406B718A
:104D2000082A44D2DFE802F00B124319242F363D43
:104D300080F86C40ECE768E080F86C20E8E713B19D
:104D400080F8704033E080F8706030E013B180F894
:104D500050602CE080F8504029E023B180F8656075
:104D600087F8036123E080F8654087F803411EE07F
:104D700023B187F8F54080F84D4018E087F8F560DA
:104D800080F84D6013E013B180F868600FE080F8A0
:104D900068400CE013B180F8666008E080F8664077
:104DA00005E013B180F8676001E080F86740521CAD
:104DB000D2B22A71082AAED398F80E102A4A8B076D
:104DC00005D587F8F16080F86460568104E087F8C3
:104DD000F14080F864405481C90702D080F829402E
:104DE00001E080F8296098F8111000F86D1FC27872
:104DF0001E48012A1ED001B3012921D04FF4805151
:104E0000A0F876101A493C200870A9F80240A9F8C9
:104E10000440B9F80210491CA9F80210B9F80210B0
:104E2000B1F5FA7F04D940F2F511A9F802102C70FF
:104E3000BDE8F08344F21C71E2E74FF40051DFE774
:104E400041F25551DCE70000FB060020A4020020DF
:104E50004801002000100140500C00209406002062
:104E6000C0040020680C0020140A0020280500203F
:104E7000F80600202DE9F05FFDF76EFA8E4D2888C8
:104E8000A5F10406C0070AD0308820F00800308061
:104E9000288820F00900288001F0AEFDD9E028889C
:104EA000DFF81892DFF81882864C80071AD5B9F817
:104EB000001041F00101A9F80010B8F80000804985
:104EC00014315030088028884FF6F9510840288066
:104ED000308840F004003080FFF784F884F83C000C
:104EE000BDE8F09F2888784F4007288871D520F0CA
:104EF00004002880FFF776F894F83C108142EFD147
:104F0000308820F004003080FDF7FEFB2078410659
:104F100005D594F84C1094F83B209142E0D03978B4
:104F2000400621F00201397004D5FEF711FB97F815
:104F30002F7004E094F83C00FDF760FA0746DFF8B4
:104F400080B140F68C2A0BF1180B062F47D294F84B
:104F50003800B8423ED03846FDF7D4F92078C00773
:104F600016D094F83A0094F8391000F003029142F8
:104F700006D0A17A00F0010001F00101884215D1AC
:104F8000FDF72AFBFBF740FFFDF752FC384689E0AE
:104F9000FDF722FBFBF738FFFDF74AFC3846FDF72B
:104FA0003BFB207840F00100207099E7288820F032
:104FB00008002880206B810801EBD000504515D2F5
:104FC000B8F800100844ABF80000308840F0080042
:104FD00003E00DE0308820F00800308080E7B9F869
:104FE000001041F00101A9F80010DFE75046E7E7A3
:104FF0000007288831D520F008002880308820F06C
:1050000008003080FEF7EEFF84F83C00FDF77CFBE3
:10501000387820F0020038702078400604D5FEF77A
:1050200097FA97F82F5004E094F83C00FDF7E6F962
:105030000546062D08D294F83800A842B5D0FDF7F1
:10504000CBFAFBF7E1FE2AE02048C18841F040019D
:10505000C180BDE8F05FFDF7CBBBC006288825D531
:1050600020F010002880308820F01000308097F861
:1050700038000C2802D2401C87F83800387840F0FD
:1050800002003870FEF764FA97F82F50787884F8A9
:10509000390094F83800A84287D0FDF79DFAFDF753
:1050A000C7FB2846BDE8F05FFDF7B6BA4EF2BE1169
:1050B0000840288014E7000010040040000400406D
:1050C000240400404801002048040020140A002065
:1050D0002DE9F04F514F85B0388820F0010038801D
:1050E0004E480026103006804D4CDFF838A14FF0B6
:1050F000010894F85C0042F63029C10774D072B6FA
:105100004948816941F400718161816941F480619C
:1051100081614FF40040FEF7CBFE444D002128464C
:10512000FBF7D0FB00212846FBF7C2FBDFF800B1FC
:1051300000215846FBF7BCFB00213E48FCF750FA23
:105140002846FBF7DBFC5846FBF7D8FC4FF4602001
:10515000CDE902068DF8056000968DF810808DF877
:10516000048069462846FBF75BFD01231A460F21A0
:105170002846FBF7A6FD01212846FBF799FB0020F6
:105180004946401C80B28842FBD328462E6001214C
:10519000FBF7D6FD28688007FCD524484C30006812
:1051A00094F85C1021F001012144A1F85000FBF7B4
:1051B00093FB62B6FEF7D8F847F69061AAF80010A4
:1051C00094F85C00401CC0B284F85C000C2822D229
:1051D00012491431A1F80080388840F0010038806D
:1051E00005B0BDE8F08FFFE7134920F00100085A31
:1051F00012490880114945F65800083908800F48BF
:1052000047F25801001F01800C4920200C3908800A
:10521000AAF80090D4E70320A070E1E7000800405E
:10522000480400202C0800400010024000240140E7
:105230000028014008000240288E0008202C014070
:105240000029018802D041F0800101E021F08001B5
:105250000180704710B50A884B88CC881A438B8828
:1052600023431A430B891A434B8989891A430A43FA
:10527000A0F8442010BD0021018041808180C180C0
:1052800001814181818170470029818802D041F0EC
:10529000010101E021F001018180704700290188AE
:1052A00002D041F0010101E021F0010101807047CD
:1052B000002930F8441F02D041F4004101E0C1F35D
:1052C0000E010180704700004B4910B5884202D1A1
:1052D0000121C41486E0B0F1804F09D047498842CB
:1052E0000DD101210220FEF705FE0021022064E01D
:1052F00001210846FEF7FEFD002101205DE0404946
:10530000884206D101210420FEF7F4FD002104208B
:1053100053E03C49884206D101210820FEF7EAFD0E
:105320000021082049E03849884206D10121102097
:10533000FEF7E0FD002110203FE03449884206D10D
:1053400001212020FEF7D6FD0021202035E0304944
:10535000884202D10121441444E02E49884202D1FE
:105360000121CC043EE02C49884202D101210C05E8
:1053700038E02A49884202D101214C0532E028490F
:10538000884206D101214020FEF7B4FD00214020D3
:1053900013E02449884206D101218020FEF7AAFDAE
:1053A0000021802009E0204988420AD1841501218A
:1053B0002046FEF79FFD00212046BDE81040FEF785
:1053C00099BD1A49884202D101210C040AE018490A
:1053D000884202D101214C0404E0164988420AD1D6
:1053E00001218C042046FEF79DFD2046BDE81040BB
:1053F0000021FEF797BD10BD002C014000040040C5
:1054000000080040000C0040001000400014004064
:1054100000340140004C0140005001400054014064
:1054200000180040001C00400020004000400140E7
:105430000044014000480140002A828901D00A430B
:1054400000E08A438281704730B5028C22F001026D
:105450000284028C8388048B22F0020224F07305FC
:105460000C882C430D8915434A882A43114DA842C4
:105470000BD0114DA84208D0104DA84205D0104DB8
:10548000A84202D00F4DA8420DD122F008054A894A
:1054900023F440732A4322F004058A882A438D8925
:1054A0001D43CB892B4383800483C9888186028472
:1054B00030BD0000002C014000340140004001409C
:1054C0000044014000480140028B22F008020A43D8
:1054D0000283704770B5028C22F010020284028CA5
:1054E0008488038B0D8823F4E6464FF6FF7303EAA6
:1054F000052535430E8922F0200203EA06161643DD
:105500004A8803EA02123243104EB04202D0104ED3
:10551000B04215D122F080064A8924F4406403EA9F
:105520000212324322F040068A8803EA0212324312
:105530008E8903EA86062643CC8903EA8404344331
:1055400084800583C9880187028470BD002C0140D6
:1055500000340140028B4FF6FF7322F4006203EA2D
:10556000012111430183704770B5028C22F48072CF
:105570000284028C8488838B0D8823F073031D437F
:1055800022F400730E894FF6FF7202EA06261E43CC
:105590004B8802EA03233343104EB04202D0104E30
:1055A000B04215D123F400664B8924F4405402EA3A
:1055B0000323334323F480668B8802EA03233343B7
:1055C0008E8902EA06162643CC8902EA0414344383
:1055D00084808583C9888187038470BD002C014045
:1055E00000340140828B22F008020A438283704714
:1055F00070B5028C22F480520284048C8288838BE2
:105600000D8823F4E6464FF6FF7303EA052535437C
:1056100024F400560C8903EA043434434E8803EA28
:1056200006362643094CA04202D0094CA04205D1BF
:1056300022F480448A8903EA82122243828085838D
:10564000C988A0F84010068470BD0000002C0140FD
:1056500000340140828B4FF6FF7322F4006203EAAC
:1056600001211143818370470185828270478288BE
:1056700022F07002828082880A4382807047A0F8FC
:105680004010704730B502881B4B1C4C98420DD01F
:10569000A0420BD0B0F1804F08D0194DA84205D0E0
:1056A000184DA84202D0184DA84203D122F070052F
:1056B0004A882A43154DA84206D0154DA84203D06A
:1056C00022F44075CA882A4302808A8882850A8823
:1056D000028598420AD0A04208D00E4A904205D0D6
:1056E0000D4A904202D00D4A904201D1097A0186BA
:1056F0000121818230BD0000002C014000340140B6
:105700000004004000080040000C00400010004071
:1057100000140040004001400044014000480140A6
:105720004FF6FF71818000210180C18041800172AC
:1057300070470029018802D041F0020101E021F008
:105740000201018070470029018802D041F0040164
:1057500001E021F00401018070470000204810B5ED
:1057600090F82010026801F01F001E4951F8200037
:105770001D490242086802D040F4803001E020F464
:105780008030086019484FF00002807941061848BF
:1057900024D4184903880C88E31A9CB201230F2CE7
:1057A00008D30C8804808468062C03DB124C247810
:1057B000022C05D0427F012A06D00988418010BD05
:1057C0004377C2770A88428042880988891A89B259
:1057D00040F635429142F2D3C37710BD427710BDF7
:1057E000D80500206C920008A4020020140A0020B2
:1057F000300C002004070020FB0600202DE9F04FAC
:10580000DFF8B8B16A48DFF8AC91DFF8ACA190F8E6
:105810000EC0BBF91A70BBF91C60BBF91850BBF97C
:105820006C10BCF1070F48D2DFE80CF08D041A3081
:10583000485E7600D9F800208284DAF80020C2841D
:10584000828CC38CA7EB820212B2A6EB83034A437D
:105850001BB2594342F3CF2241F3CF23D11870E05A
:10586000D9F800204284DAF80020C284428CA5EBEB
:10587000820213B2C28C4B43A6EB820212B243F3F4
:10588000CF24514341F3CF23E11814E0D9F800208D
:10589000C284DAF800204284C28C438CA6EB8202D8
:1058A00012B2A5EB83031CB24A43614342F3CF23F8
:1058B00041F3CF24191949420AB244E0D9F8002033
:1058C0008284DAF800204284828C438CA7EB820227
:1058D00012B2A5EB83034A431BB2594342F3CF22D2
:1058E00041F3CF24111914E0D9F800204284DAF8EA
:1058F00000208284428C838CA5EB820212B2A7EB3B
:1059000083034A431BB242F3CF24594341F3CF22CE
:10591000A11849420BB216E0D9F80020C284DAF887
:1059200000208284C28C838CA6EB820212B2A7EB89
:1059300083031CB24A4342F3CF23614341F3CF2296
:10594000991849420CB2BBF91E50594605F21E5631
:10595000A64201DACE8306E0A5F21E55A54201DD7E
:10596000CD8300E0CC83B1F9204004F21E5595426E
:1059700001DA0D8406E0A4F21E54944201DD0C8489
:1059800000E00A84B1F9222002F21E549C4202DA9D
:10599000ABF8224008E0A2F21E529A4202DDABF8B8
:1059A000222001E0ABF82230417B8173BDE8F08F0B
:1059B000A40200203C2401403C280140280500208E
:1059C0002DE9F04704465748584D002602785648BE
:1059D000022AB0F9301004D0082A7DD0092A07D055
:1059E00008E0C27B022A02D1B0F8402032B1E18740
:1059F00069812E8184F83C60BDE8F0874C49DFF86E
:105A00003481496A0F14E7808068410210D5B4F9E7
:105A1000020040F2DA21884269DD40F26A418842A0
:105A20003FDCA0F2DA20FAF7FAFC0022424B4BE00E
:105A3000C0F3C001C0F30020DFF8009181420CD117
:105A4000D8F8440040F2BA41884250DD40F66A116D
:105A5000884226DCA0F2BA4032E039480078C0061D
:105A60000CD5D8F8440041F2243188423FDD41F2A0
:105A7000D471884215DC00F6DC401FE0314890F814
:105A80007010012903D090F86F0001282FD1B4F9CC
:105A9000020041F6C811884229DD41F6786188424A
:105AA0000ADD0823B4F93E101A460020FEF704FF71
:105AB000E087002819DB1BE000F5C760A0F5005067
:105AC000FAF7ADFC00224B46FAF715FC0E22FAF766
:105AD00081FCFAF7DBFC00E01FE000B2C0F580407B
:105AE00078438013E087002F02DCE68700E0E78739
:105AF000E08F154FE880D8F844107964A7F84C007F
:105B000000F076FBB7F84E00688198F80A0000288C
:105B1000388F00D1404228816CE70C48B0F8700003
:105B2000688166E7FB060020A40200206C000020CC
:105B300028050020480100200000794000C0924064
:105B4000DC060020680C0020B8080020280A00208D
:105B50002DE9F041B1F9025000232B241522854292
:105B600003DAB1F90000BDE8F081B1F9AE50854229
:105B700002DDB1F9AC00F6E701EB8205B5F90250A0
:105B8000854201DD134600E01446E21852085D1C10
:105B9000AA42F1D101EB8206B6F90230834206DA5D
:105BA00036F9025C36F9044C31F9221006E01D4644
:105BB00031F92240B6F90630B6F90410401B091B32
:105BC000C6178911B60346EA90468703A1FB070C66
:105BD000CA1702FB07C201FB06215A1BD317FAF7AB
:105BE000A3FA000A40EA0160001900B2B0F5804F44
:105BF000B9DB43F6FF70B6E770B5134C40F22445AD
:105C00002946204600F03EF800281BD0204600F030
:105C1000C7F82946204600F01DF80C4C002120460C
:105C2000FBF7DEFC2046FBF759FDC0F16400084994
:105C3000C0B20428087201D900F046F9BDE87040EE
:105C4000FBF792BD70BD00000038014058000240D3
:105C5000640600200A0A01219140C943018070476F
:105C60000029818902D041F4005101E021F4005162
:105C700081817047002A828A01D00A4300E08A436A
:105C80008282704730B501F01F0201240025C1F364
:105C9000421304FA02F2012B0FD0022B0FD0838A99
:105CA0004FEA11210088134204FA01F400EA0400CB
:105CB00001D000B10125284630BD8389F0E7038A71
:105CC000EEE710B5C1F3421301F01F040121A1401A
:105CD000012B07D0022B07D01430002A026805D010
:105CE0000A4304E00C30F8E71030F6E78A4302601C
:105CF00010BD000030B50446008A85B00D464CF654
:105D0000FF710840E98801432182A1894EF6F31012
:105D10000140A8882A8910436A890A431043A08158
:105D2000A08A4FF6FF410840A9890143A182684635
:105D3000FEF704F91948844201D1039800E0029863
:105D4000A189090400EBC00101EB0010296801D50D
:105D5000490000E08900B0FBF1F06422B0FBF2F1F1
:105D600009010B096FF018056B4300EB8300A38951
:105D70001D044FF0320306D503EBC000B0FBF2F078
:105D800000F0070005E003EB0010B0FBF2F000F0BC
:105D90000F000843208105B030BD000000380140ED
:105DA0008088C0F308007047F8B501210920FEF78C
:105DB000ADF801218803FEF7A9F810258DF80350EE
:105DC0002020ADF800001A4E03248DF802406946E9
:105DD0003046FCF709FA16490C31086820F020001B
:105DE000086018208DF803004020ADF800008DF801
:105DF000024069463046FCF7F7F948208DF8030069
:105E00008020ADF8000069463046FCF7EDF98DF8CA
:105E100003502801ADF800008DF802406946304675
:105E2000FCF7E2F901210420FCF730FAF8BD00008C
:105E3000000C014030B585B0FFF7B6FF00244FF4E9
:105E4000E1300090ADF808400C201D4DADF8044045
:105E5000ADF80A00ADF80640ADF80C40694628469A
:105E6000FFF748FF25208DF8100004208DF8110061
:105E70008DF8124001208DF8130004A8FDF704FDF1
:105E8000012240F224412846FFF71BFF012128464A
:105E9000FFF7E6FEFBF792FC012280212846FFF780
:105EA000E9FE012240212846FFF7E4FE01220221FB
:105EB0000448FBF727FCFBF781FC05B030BD000070
:105EC000003801404400024070B51D4D0024287880
:105ED000432834D16878462831D1A878502807D093
:105EE000512805D0812803D0892801D0212826D126
:105EF000144E7071E9787172A81C891CFBF754F874
:105F0000B072717A294409793182884217D106F139
:105F10000E00017841F0020101700B48016841F068
:105F200020010160317A0948002204E02B5D03550D
:105F30002A55641CE4B28C42F8D38078707170BD2D
:105F400090070020640600200C0C01409A0B0020F2
:105F500070B51D20FDF777FCFDF7FAFA1D20FDF75F
:105F600088FC154890F82F10144D0623144C85F822
:105F7000381090F83B1095F83B201143012A04D0CB
:105F8000022A07D0042A0AD010E0827A8A420DD071
:105F9000007B09E0027D8A4208D0807D04E0827F98
:105FA0008A4203D090F82000884200D1237000205C
:105FB00085F8400070BD0000480400204801002022
:105FC000FB0600200B4800214180A0F1B0018A8926
:105FD0008280CB891A44C2800B8A1A4402814B8A80
:105FE0001A444281898A1144818143F6FF71C1813B
:105FF00070470000F8010020084940F61C72B1F912
:106000000C00904202DA00F59F7005E041F2E302D5
:10601000904201DDA0F59F70C88170476C000020A0
:1060200038B51348C16941F00401C1611E208DF8E3
:10603000000002208DF801008DF8020001248DF887
:1060400003406846FDF720FC0A498420088009497E
:1060500047F690602C3108800020091F0880054910
:1060600014310C80091F0880081F048038BD00000F
:10607000001002400008004030B420491E4A457814
:106080008B7A114692F83B4091F83910AC4218D106
:106090004BB10379994202D04379994201D14079B9
:1060A0001AE0807909E08379994202D0C479A1424B
:1060B00002D182F82F3011E0407982F82F0030BCF5
:1060C0007047C578AC42FAD16BB1C379994202D01E
:1060D000037A994205D1007A82F82F0030BCFEF78E
:1060E00081BC407AE9E7437A9942E2D00479A1423F
:1060F000DFD0007AE1E700004804002048010020DA
:10610000FEE700002DE9F0470446007F012868D132
:106110003548E1880288511A89B2072916D30088C8
:10612000E080B4F9000044F2DD414843401346F6F4
:10613000D96148438013A060401000B2A0814FF0A5
:106140008051B1FBF0F0FAF765F92061B4F90C6009
:1061500096B1B4F902104DF6B05048430014A08235
:10616000B4F904704DF6B05207FB02F24FEA224533
:10617000E58204D4024603E00020E08330E042429E
:1061800012B22283002D01DB2B4600E06B421BB2D2
:10619000DFF85890638398464FF4804AB24208DA99
:1061A000FAF72FF92169FAF702F8FAF756F980138E
:1061B00004E0002901DA484600E05046E083B0459B
:1061C00009DA2846FAF71DF92169F9F7F0FFFAF71D
:1061D00044F9801304E0002F01DA484600E05046FD
:1061E0002084BDE8F08700000407002000C0FFFF06
:1061F00010B52848294C01782748022905D1C17BD0
:10620000022902D1B0F8401029B1008EA4F84E0046
:106210000020208710BD90F8462020482049022AFF
:10622000B0F84400097800B2C1F3810103D0012A1B
:106230000CD01C4913E0012904D0022904D01949CB
:106240006C390CE018490AE0184908E0012904D02B
:1062500002291CD015496C3101E013496C31FBF760
:106260000FFE0E49A4F8400080B2483101F092FAC6
:10627000B4F94C00B4F94A2041425143891324F83F
:10628000381FB4F9101048438013E08210BD07494D
:106290006C39E4E7FB060020A4020020B8080020C7
:1062A000C0040020BE8C0008368A00087A8B0008E3
:1062B0000348002180F82A10C1830187704700003D
:1062C000B808002010B504000B462D4AC3F10000A9
:1062D00028D56442002B12DAA04207DA214600F0EA
:1062E00027FA32F81000C0F5404041E00146204650
:1062F00000F01EFA32F8100000F5004038E0A3422A
:1063000008DA2146184600F013FA32F8100000F5BA
:1063100040402DE0204600F00BFA32F81000C0F5A6
:10632000803025E0002B12DAA04207DA214600F087
:10633000FFF932F8100000F5804019E001462046D0
:1063400000F0F6F932F81000C0F5004010E0A3426A
:1063500008DA2146184600F0EBF932F81000C0F5D3
:10636000804005E053B1204600F0E2F932F8100019
:10637000B0F5004F01DDA0F5803010BD002010BD4C
:10638000348E000840438013494300EBA1300022C3
:106390000302002B14DDB3F5001F01DC802001E0B7
:1063A0004FF4005093FBF0F1014401EBD17149101F
:1063B000814206D0521CD2B20846062AF2D300E02F
:1063C0000021C80000B2704702E008C8121F08C1CF
:1063D000002AFAD170477047002001E001C1121F66
:1063E000002AFBD1704700002DE9F047A44CA548D6
:1063F00021880288511A89B20F297DD30088A4F11F
:106400003C052080288F08B1401E28872B789E4AA3
:10641000C3F3810001281DD0022820D0D18B9848D9
:106420009A4FDFF86C92407E0026B1F5926F1DD82E
:10643000142819D378206076F88840F01000F8808E
:1064400040F26660A88123F001002870D67389F8B5
:10645000006015E0D08B00EB4000C00302E0D08B61
:106460008C494843010CDAE7401C04E0B1F5DB6FCE
:1064700006D310B1401E607602E043F001002870A0
:10648000B5F90200B5F914304143C3EBC303C1F3BE
:106490008F31C3F3D10303EB510109B2A9829046B6
:1064A000D28B4FF080535043B5F91620C0F38F3094
:1064B000C2EBC202C2F3D10202EB500000B2E8828A
:1064C000AA6A42431213EA6293FBF2F22A63724A07
:1064D0001080A2680A44A260E1680144E160207C67
:1064E000401CC0B22074072806D942F3CF0028838D
:1064F000C9106983E66000E0BFE0A66041F6C8010C
:106500002674884204DD298B644AB2FBF1F1E981EB
:10651000C117890341EA9041800342F69B42002360
:10652000F9F702FEA88456482A78A0F13C005C499D
:10653000B0F90600930700FB01F14FEA2141C2F3D5
:10654000810215D5012A07D0022A0BD04FF26851DB
:1065500041430914A18011E049F68C4250430014D4
:10656000A0801FE04CF6183141430914A18025E0BA
:10657000012A0DD0022A17D0A080698449494843D6
:106580000014E083FBF79CFA47480088C0B143E061
:106590004AF65C3242431214A2804BF62C2250433E
:1065A00000146884E183EDE74DF2AC5141430914D6
:1065B000A1804EF27C414143091469843B49DEE7E6
:1065C00095F8200000BB88F80F6089F80060B5F9E5
:1065D0001A00A0F50C519F39B1F56E7F18D8617F74
:1065E000F42912D93249E8802E4AA1F846005043D6
:1065F0000014A880A1F84400FF2085F8200081F84D
:1066000028002C493C20087006E0491C617703E013
:10661000607F08B1401E6077B5F91A10B4F91E000A
:1066200081420EDDA07E7D2809D9F88840F008005F
:10663000F8802148017821F0020101700EE0401C31
:1066400006E0A0F23D10814208DAA07E10B1401EA3
:10665000A07603E0F88820F00800F880B5F918105B
:10666000606908446061217E491CC9B221761F29F6
:1066700003D94011A88366612676BDE8F087000043
:10668000FC04002004070020A4020020140A0020BB
:10669000FB06002030330100C809002074E8260BF7
:1066A000CC0E01004885010006070020D0450100FE
:1066B000680C0020F8060020D2050020024941F6AF
:1066C0008B30886270470000C004002070B5164C03
:1066D00006252078062825D2DFE800F003080E14EE
:1066E0001A211248FAF79EFC012016E00F48801D7F
:1066F000FAF798FC022010E00C480C30FAF792FCF4
:1067000003200AE009481230FAF78CFC042004E068
:1067100006481830FAF786FC0520207070BDFAF79D
:10672000A1FC2570257070BDFC0600202A8D000894
:10673000090A05D0B0FBF1F0FF2800D9FF2070470F
:1067400000207047D0E90021C368521A5A4301EB78
:10675000A231816041607047B0F90020B0F90210A9
:10676000B0F90630521A5A4301EBA23181804180C0
:1067700070470000F0B54F4C20884F49504E514BA8
:106780000A8B801A82B24D480F2A057801F1580011
:1067900032D322880A83197A5FEA017C0146B1F973
:1067A000021001F1020217B2A1F1020212B20BD5DE
:1067B000022D01D044490FE0DFF810C1BCF900C040
:1067C000614513DC17DB13E0022D15D1D6F844C068
:1067D000BCF5FA5F03DC3E49098841800CE0DFF834
:1067E000F4C0BCF900C0614505DB01DD428003E077
:1067F000A0F802C000E04780018F2288A2EB0101CF
:1068000089B29C2941D321880187996A0022B1F578
:10681000804F2CDBB16CB1F5405F28DD2E4940F292
:106820006664B1F91010A14211DD43F69914A1423A
:1068300002DB40F2333108E040F23334A1F266610A
:10684000614343F2333491FBF4F1818700E08287A6
:106850002249B3F806410978C1F381011CB1818F47
:1068600001F21E5119E093F84630022B0ED08287B8
:10687000022D00D08287B0F95410B0F93C2001F10C
:10688000140393420BDAA0F85430F0BD012901D073
:106890000229E4D1818F01F233318187E8E702F1E7
:1068A0001403994203DD1439A0F85410F0BDA0F888
:1068B0005420F0BD0407002014000020FB06002037
:1068C00048010020A4020020BE040020BC040020D7
:1068D000BA040020B804002028050020C0040020CD
:1068E0002DE9FC4101210220FDF7F8FA01211920D0
:1068F000FDF70CFB01213C48FBF7C8FC4027ADF835
:10690000007003248DF802400420384D8DF80300F8
:1069100069462846FBF768FCE001ADF800008DF8F9
:1069200002401C208DF8030069462846FBF75CFCFA
:106930004FF4E0712846FBF7DEFCA815ADF8000027
:106940008DF8024010208DF8030069462848FBF7B7
:106950004BFC4FF4A060FCF7C9FF1D208DF804002C
:1069600001268DF8056000258DF806508DF807602A
:1069700001A8FCF789FF1F498C2008801D494FF6AC
:10698000FA702C3108806E20091F088019481430D5
:106990000680184808300780164920310D80154AB6
:1069A000D020121D1080134A45F2F30018321080D7
:1069B0000A1F45F2500010800E4A4FF6FF70383221
:1069C0001080121D1080121D108041F21B100880D3
:1069D00000F012F8FBF70CFF064810300580001F8E
:1069E0000480BDE8FC810000000C1A00001001408A
:1069F000000C01400004004070B51D20FCF718FF9A
:106A00002A4D40212846FBF76DFC84008021284652
:106A1000FBF768FC44EA4004A9152846FBF762FC32
:106A20000443E0B2224C84F83C00FBF7E7FC054647
:106A3000052805D91F48C18841F04001C18001E007
:106A400084F838501C48007A000703D594F83800C1
:106A50001A490D5C4FF6FA702063E062A062606232
:106A60002062E061A0611648606300206064A06459
:106A700084F83F0084F84000FBF76EFCA07AFF2802
:106A800011D0022084F83D000E4800882066284678
:106A9000FCF710F9207820F001002070BDE870406C
:106AA0001D20FCF7DBBE0120ECE7000000100140D8
:106AB00048010020140A0020A40200203896000893
:106AC000DCFF0500240400402DE9F0434E484F4907
:106AD00002880B889A1A92B20F2A69D3098801801A
:106AE0004B49098B027D00EB42029180017D491CDC
:106AF000C9B2017508295BD3002404752246017DC3
:106B000000EB4103491CB3F90430C9B202EB630244
:106B100012B201750829F2D33E4904753E4B4A80F2
:106B200044800E789D895FEAC67C40F638694FF054
:106B3000030714D0A2F22B5C42F6E858C44520D3D8
:106B4000A1F1020C26F00204ACF8002047750C708D
:106B500040F22B54A24211DA45F004021EE046F046
:106B600001060E704A4507DD45F001029A8126F0C4
:106B700002020A70477519E0447517E045F00202F9
:106B80000CE04A450CDA8775427D12B1521E4275FF
:106B90000CE046F002020A7025F007029A8105E037
:106BA000B30703D5837D2BB15B1E83754088888036
:106BB000BDE8F08342F6AA239A4222DAB1F9043002
:106BC0002BB941F2CD05AA4201DA4480EEE7134C1D
:106BD000920302EB843241F67244B2FBF4F214B237
:106BE00040F2333502464480AC4200DA5580B2F9B7
:106BF0000240E41A04F5A374B4F5237FD6D8438089
:106C0000D4E74FF48043FAE79C0A002004070020F1
:106C1000A4020020D2050020140A0020C8F1FFFFC2
:106C20002DE9F0416C4CDFF8B4E14FF0000594F829
:106C30002810C80706D094F92C104B42002956DDC5
:106C40000E4655E0664884F82B50E586654A90F874
:106C5000380084F834001586CEF80450CEF8085079
:106C6000614E40F26663CEF80C50A4F8703036F8EE
:106C700010005E4E768830444FF6FF7606EA8000BC
:106C800024F8240B4FF080602060A32020846084CF
:106C90005810A084E38440F6991020855800608540
:106CA0004FF48050A08541F23330E08541F26660B8
:106CB000208641F69910608641F6CC40A0864FF4BC
:106CC0000050E08642F23330208742F266606087EF
:106CD00042F69910A08742F6CC40E08782F89D509A
:106CE00041F00100207184F84450BDE8F0811E4657
:106CF00094F92B004242002801DD074600E01746C8
:106D0000F61B012E0BD0002800DB02465FFA82F64C
:106D100084F82C0094F84300012805D041E00029B4
:106D200000DA1946CEB2F3E794F92D305942002B20
:106D300001DB184600E0084694F92E20C7B2504205
:106D4000002A01DB944600E08446BC4508DD002AA9
:106D500000DA0246D7B2002B00DA0B46D8B207E0C1
:106D6000002B00DA0B46DFB2002A00DB1046C0B26F
:106D700004EB4000B0F9441004EB470030F9442F15
:106D800011444910018084F8435084F8325084F84B
:106D9000315084F8305084F82F5084F82E5084F805
:106DA0002D5004EB46007546B0F94400E086BEF86D
:106DB0000410C82309B26422FDF77EFD6860E9680B
:106DC000401AA9680844A860B5F900104843C013E8
:106DD000E860A4F8700088E7280A0020C0050020B9
:106DE00048010020A40200204A9600086C00002000
:106DF0002DE9F0415F4C94F82800C00779D05E4837
:106E000094F83410002690F838005C4D814271D01F
:106E10005B4AA4F866605B4F535C2246834292F95A
:106E20002B2002D07B5C83420FD1521C52B284F8DB
:106E30002B20795C814202D1521C84F82B2094F9DA
:106E40002B100F291BDD0F2117E04F4B5F5C4F4BC1
:106E5000874202D05F5C874211D1521E52B284F841
:106E60002B20595C814202D1521E84F82B2094F9C8
:106E70002B206FF00E018A4201DA84F82B103D4975
:106E800094F833302D3194F82B205A5494F8331061
:106E9000491CC9B284F83310062901D384F8336041
:106EA00094F92D2094F92F108A4211D194F93120B0
:106EB00091420DD194F92E2094F930108A4207D1D5
:106EC00094F93220914203D1012184F8431001E06A
:106ED00084F84360284984F8340094F92B30097809
:106EE000012B0DDD254A4F07926804D542F00802B8
:106EF00003E03CE015E022F00802AA6084F82900D3
:106F0000B3F1FF3F0ADA4907A96802D521F0080169
:106F100001E041F00801A96084F82900FBF71CFAA0
:106F200011E094F8430001280DD1B4F8660043F64F
:106F30000951401C80B2A4F86600884203D9A4F825
:106F4000666084F84360E87B082810D0B5F93010FB
:106F5000512341220020FDF7AFFC2886002806D1EE
:106F60000B48067014F8280F20F001002070BDE8CF
:106F7000F0810000280A002048010020A40200201F
:106F80002C960008329600083E96000844960008A9
:106F9000FB06002030B52049204AB1F86A3010883D
:106FA000C01A80B20F2836D31088A1F86A001C4D91
:106FB00000204FF000432A5C940903D00124B4EB75
:106FC000921F24D1D20622D0164A52F820201268ED
:106FD000134C123434F81040224201EB000494F9AF
:106FE000722008D00A2A04DB0A6823FA00F422433C
:106FF00008E0521C09E012F10A0F05DC0A6823FAC6
:1070000000F4A2430A6002E0521E84F87220401C81
:10701000C0B21128CFD330BDD8050020040700200E
:1070200038920008389300082DE9F00779497A482A
:107030000A8903889A1A92B2082A74D300880881B0
:10704000A1F12C0042890AB1521E4281734A92F882
:107050002820802A67D302F03F020A70C2890AB151
:10706000521EC281B1F90620902A0CDB8A46FF2A03
:1070700009D08146C089002855D16948002300788D
:10708000092805D005E0BDE8F007624800F092B994
:107090000823644A92F8EA500DB143F004036248B1
:1070A000817AC90701D043F00203D2F808C05FEA31
:1070B0000C5101D543F00103176800215B4EFC031E
:1070C00002D596F8654004B18021C4885FEA44681F
:1070D00001D541F040015FEA845801D541F020011B
:1070E0005FEAC47801D041F01001007A400701D571
:1070F00041F008014E480078C00701D041F004017A
:10710000A00601D541F001010020012D00D1082089
:1071100096F8705085B992F84620022A04D0012AC8
:1071200005D03AB108E072E040F0030004E040F01E
:10713000020001E040F001007A0701D440F0200095
:10714000CCF3C0020025CCF3002C624502D13A07F3
:1071500000D4042596F86F20012A01D145F00105DD
:10716000344A0027BC4612783E46C2F38102012A07
:1071700004D0022A04D0032A04D004E0022602E04C
:10718000042600E010262C4A64060ED5214C1C343F
:107190002478240609D51478640606D4274A40F6D4
:1071A000CC44926D6243140C05E0B2F8AE2040F678
:1071B00099146243940B4FF008088AF80A804FF044
:1071C00061088AF80B808AF80C308AF80D108AF86A
:1071D0000E008AF80F508AF81070270A4B4083F08F
:1071E0006901414069408AF8117079408AF812407B
:1071F000614052468AF813C071408AF81460517594
:107200004FF4C871A9F80E10FF20AAF80600BDE8D7
:10721000F0077047C006002004070020D8050020B2
:10722000FB060020A4020020140A0020680C0020A5
:107230000C090020C004002048010020F4070020B1
:107240004C48816941F0FC0181614FF4A060FCF77A
:107250004DFBFBF75BFBFCF7B5FCF9F7A7FCFCF774
:10726000A3FAFDF72FFAFFF73BFBFCF7E3F9FFF773
:10727000C3FBFBF7BDFA404D4FF40050A5F81601D3
:10728000FEF7D8FD00214FF4FA5340F2EE22002021
:10729000401C80B29842FBD3491C89B29142F6D37C
:1072A0003648002680F87260F9F716FBF9F7B0FF50
:1072B000FCF7B8FCF9F784FEFEF7B2FE1022304965
:1072C0003048F8F762FF304C314FE08820F0400042
:1072D000E0802E48017821F020010170FA20F88129
:1072E0004FF49670E887FFF7E9F92A492A48FCF736
:1072F0000FFC2A48FCF738FC2948416A884729488E
:10730000416B8847FEF7D4FF27494220C8802749B0
:10731000C8603E71E088E0812089208260896082B7
:10732000FAF7DAFEFAF73CFEFFF75EF8FFF7CCFB60
:1073300000F0F8F9FFF72EFE01F0F2F8FEF70EFA72
:10734000FAF78EFCFBF7D4FCFFF714FAFCF7C4FE47
:10735000FBF7F6F8FBF728F900F07AF8FFF764FE80
:107360001348FAF775FA00F06FFAFDF7EFF9FAF73C
:10737000D9FBCFE700100240A4020020280500201E
:10738000680C002018060020140A00204801002084
:10739000F806002094080020700800200404002053
:1073A00040000020DC0000202007002034040020E2
:1073B00094090020F0B523490278B0F90640002373
:1073C0001F4E31F81210FF2C18D0B0F904701E4D6A
:1073D000BC4231DA00EBE40704F00704BF7AA740AF
:1073E0008478FFB23CB190F801C0ACF1010C644567
:1073F0001FDA3C061DD455F822200DE056F8222055
:10740000116012498A79521CD2B28A71022A02D3BF
:107410008370C3808B71F0BD11608178491CC9B243
:10742000817042789142F6D38370C188491CC18033
:10743000F0BD56F82220EFE755F822201160F4E75E
:10744000189400084A920008C0930008940600208F
:10745000F0B561486149B0F86C200B889A1A92B275
:107460009C2A7BD30988A0F86C105D495D4F91F888
:107470002A1001F0070297F84610022A00D1491E8F
:10748000594C80F83E104FF00203E2884FF00001A3
:10749000550401D5012236E0A489E50601D506226E
:1074A00031E0250701D508222DE0550603D44F4DC4
:1074B0002D78AD0601D5042225E0150501D507225A
:1074C00021E0150601D50A221DE0950601D50C2202
:1074D00019E0150701D50B2215E0550701D4D50594
:1074E00001D510220FE0D50601D505220BE0650776
:1074F00003D4A50701D4E40702D080F86E3007E07A
:10750000920403D5032280F86E2001E080F86E100B
:10751000374A384C92F820E0324A251FD2F808C08A
:107520002D4AB2F87060721C92B2BEF1000F0DD0FD
:107530002CF4000CC7F808C090F86E70B7B11E2F7D
:107540001AD090F86F200AB325E007E04CF400064B
:10755000BE60A0F870200A2A01D22360F0BD142A70
:1075600001D22B60F0BDA0F87010F0BD2B60A0F828
:10757000701080F86F10F0BD642E04D2A0F8702057
:10758000322AEED3E9E7A0F87010EAE77F1C80F812
:107590006F70A0F8701090F86F20012A10D0002AA8
:1075A000E9D0B0F87060761CB6B2A0F870601E2EFC
:1075B000D7D323603C2EDED9521E80F86F20D2E74D
:1075C000B0F87020521C92B2A0F870202360C82A34
:1075D000D1D980F86F10C6E7D80500200407002035
:1075E000680C0020A4020020140A0020480100209A
:1075F000C0040020141C0140F0B54248B0F8481007
:10760000491C89B2A0F8481002297AD33E490024C7
:10761000A0F848400A783D4B042A57D04FF48041E7
:10762000082A0BD0A0F10C02B2F900208A4200DA3D
:107630001146B3F980208A4200DA1146344A926931
:107640008A4200DA11B2418282881D8AC2EB850229
:10765000304D12B22D78C5F381062A4D42F2AA466A
:107660007243B5F9765092126A431213C26086686B
:107670001546C6EBC60642F3D102F60202EBA6326D
:107680008260C66C1644C664B0F850707F1CBFB2EE
:10769000A0F85070B7F5806F04D3B6120682A0F838
:1076A0005040C464891A1C4EC26A724340F2555657
:1076B0004E4302EB4602466A32444262B3F930302E
:1076C000B2EB034F06DD1A04426206E01349B1F93A
:1076D0000410B3E7002A00DA4462C162104990F84E
:1076E0003D2091F838108A420BD080F83D10B0F858
:1076F0004210A0F84410B0F84010A0F84210A0F8D2
:107700004050F0BD28050020FB060020A402002008
:10771000000C0020C0040020C3F5FFFF1C0C00205B
:107720004801002017481849B0F85A200B889A1AC7
:1077300092B20F2A25D30988A0F85A10134941F6AE
:10774000515391F84D10CA0701464FF48042B1F9E8
:10775000001059438913A0F86C100D490B78A0F163
:107760000C01022B06D1B1F90030934202DA1B1D45
:107770000B8000E00A800021A0F8601020F85C1F58
:10778000428070472805002004070020680C002074
:10779000FB0600204FF6FF7202EA800210F440431D
:1077A00015480ED0B3F5804F14D0B3F5004F4FEA13
:1077B000122216D0C2F5807330F813305B424B8032
:1077C00005E0120A30F812304B80C2F5807230F8B2
:1077D00012000FE0120AC2F5807330F813304B80AC
:1077E00005E030F81230C2F580725B424B8030F811
:1077F000120040420880704734900008104A518AB5
:10780000908AD28A16384639A2F1110200D549422F
:10781000002A00DA52421144002800DA40420844AB
:10782000084943F6284300B2B1F936205A4392136F
:1078300040F2D733584302EBA030C88670470000AF
:10784000A402002028050020F0B5904990480A893C
:1078500003889A1A92B23E2A1ED30088088101F149
:1078600038004FF4FA63428A9A4202D2521C428292
:1078700000E04382874A92F82220802A0CD302F04B
:107880003F020A70B1F90620402A06DBFF2A04D025
:10789000C2883AB1521EC280F0BDBDE8F0407B48BC
:1078A000FFF788BD428A9A42F6D307784FF0010E5F
:1078B0003A074FF0FF055BD5847A40F2DC5263074C
:1078C00008D444F004038372C28081F80BE081F88D
:1078D0000AE04CE04378072B05D0032B03D0052B9F
:1078E00001D0062B07D1660605D444F0400383720D
:1078F000C280052239E0654A5FEA437C02F1380222
:107900004FF42076127A0DD55FEAC26C0AD45FEA92
:10791000446C07D442F0100202723A0628D4C680A2
:10792000192222E0DF0709D0970707D4670605D49C
:1079300042F002020272C680042216E09F0709D5B7
:10794000170707D4670605D442F008020272C68002
:1079500003220AE01B070BD5530709D4630607D49B
:1079600042F004020272C6800B22CA728A72CD8073
:10797000494AB2F92230B2F91A7003F23D140022DA
:10798000A74200DB0276414E444C06F13806A4794A
:10799000B6895FEAC46C06F101064FF4C874B6B24A
:1079A00013D58681B6F57A7F05D9017A21F0800159
:1079B00001728281F0BD037A1E06FBD4828143F0FE
:1079C00080020272C480112035E09F4216DA037EE5
:1079D000052B13D28681B6F5487F04D98281027ABD
:1079E00022F040020272027A5606E3D45B1C037650
:1079F00042F040020272C48002201CE0284B1C8925
:107A0000C4F3C006C4F3002740F2EE24BE4216D1F0
:107A10001E78360713D4427E012ACBD1428BB2F5B1
:107A2000167F02D2521C4283F0BD827A42F00202DB
:107A30008272C4800F20C8728872CD80F0BD93F826
:107A40000D714FF40046012F18D1164F41F6583CE6
:107A50007F6C674512DD83F80CE1134B1E60C38A0F
:107A6000A34202D25B1CC382F0BD4FF4FA73C38001
:107A70001C23CB728B72CD80C282F0BDC2820A48B9
:107A800083F80C21001F0660F0BD0000A406002052
:107A900004070020D8050020C0040020140A00209C
:107AA000A402002048010020140801402DE9F05FE5
:107AB000FE48FF49DFF8FCA3007E0A1D131D0128C4
:107AC000504650D030F85A4F0C8041881180BAF897
:107AD0005E001880FDF792FEF74DF84C49F2CD326A
:107AE000B5F91E006083B5F9201043F6CC4C00EBCD
:107AF000410151430914A183B4F92230B4F9206043
:107B000001FB03F200FB062242F38F326282B4F9DA
:107B10001670714307FB0CF7BF1340F2333C02FBB6
:107B20000CF207EBA23200FB1310E54FE282801348
:107B3000E44EA082786C3060316930468847E24973
:107B4000308948800846FDF73BFFDFF88093012627
:107B50004FF0000B99F8000008280CD0618E2182AC
:107B600004284CD01AE030F8604F0C804188118016
:107B7000BAF86400ADE7D64890F92B10491C0229E9
:107B80003BD890F8681019B1B4F85200208205E093
:107B9000618E2182A4F8521080F86860B4F9141044
:107BA000B4F90A00CB4AF9F76DFCE062BAF9161194
:107BB000884204DDC748E162027A91400162BF4811
:107BC00047F2A3015838DFF810E390F800C04A00EC
:107BD000BCF1000F2ED0BCF1010F51D080F800B0E5
:107BE00099F8000004280DD0BA4AB4F91610B4F977
:107BF0000800243AF9F746FC07E0608EC6E7686A99
:107C00000014E062B87A70B3B448B54FA06238602F
:107C1000E06A78603846FCF7C5F8AE4D387C383DF0
:107C200001285FD0A06A2860AE480178C9075DD0FE
:107C300040695CE0B5F91EC08C44944509D8B5F99B
:107C400020C08C44944504D8B5F92250294491426F
:107C5000C6D9A0F804B0B7F8AE205946B2F5C87F2F
:107C600002D8467007E03AE0B2F5487F01D8022218
:107C700000E0032242708AF80F1089F8001025E016
:107C800080F800B0B5F91E80DC468844904509D8DC
:107C9000B5F920808844904504D8B5F9225029448C
:107CA00091429DD9B7F8AE10B1F5C87F01D84670A2
:107CB00006E0B1F5487F01D8022100E003214170C0
:107CC000A0F804C08AF80FC089F800C0BEF80610FA
:107CD00041F40061AEF80610FAF754F980E74FF46A
:107CE000AF7092E778692860B86900E0E06A686080
:107CF00078483838FCF7CAF9704C704934F8100FDE
:107D00003C39FFF747FDDFF8B491DFF8DC81A9F1DA
:107D10005809D9F81C10C9F87810B4F91010A868DF
:107D2000B4F9123000FB01F7EA68584302FB1375FF
:107D300045F38F3702FB010040F38F35A786E586B8
:107D4000A8F802704446A8F804504046FEF7DAF955
:107D5000207F09F12004012833D068424DF6B35149
:107D600040104F4360803A1422804946A9F80E50D3
:107D700083180B82801AA9F812008AF80CB0B9F99E
:107D80000EC0D84651464846BCF1000F00DD0E73C8
:107D9000B0F91020002A02DD0B7B9B1C0B73B0F99D
:107DA0001230002B02DD0D7B2D1D0D739AF80C1087
:107DB000D146072923D2DFE801F0221736141D1916
:107DC0001F00B8F920304DF6B35258424010608081
:107DD000B8F91E1051430A1422804946A9F80E3002
:107DE000C6E789F80D600AE0022100E0032189F866
:107DF0000D1004E0042500E0052589F80D502F49F9
:107E00003A4D3B4F097801290FD099F80D1040F6F3
:107E10007E5A41F6FF2B07296CD2DFE801F06BFD9B
:107E2000FCFBFAF9F8000625E7E799F80D004E4645
:107E30000728F1D2DFE800F05E0422718EB7D70088
:107E400011466046FBF74AFE2060B4F90200B4F91F
:107E5000001043F2046201445143090C26F85A1FF2
:107E60005043000C7080A6F8048000212846F8F7E3
:107E700071FE00213846F8F76DFE80E1504201B2F4
:107E8000584200B2FBF72AFE2060B4F9020043F228
:107E900004614143090C26F85A1FB4F90010084444
:107EA00043F204614843000C708024E094090020F0
:107EB000342C0140A4020020280500206C00002082
:107EC0004801002034040020F4030020FB060020B9
:107ED000280A002094080020140A0020A2FEFFFFB8
:107EE000EC0900200C090020C809002000240140F2
:107EF00000280140B0E0A6F8048000212846F8F7E9
:107F000029FE00213846F8F725FE92E12846F8F7C9
:107F1000ABFE01231A46072193E061461846FBF7A2
:107F2000DDFD206026F85A8FB4F90200B4F9001084
:107F300043F2046201445143090C71805043000C28
:107F4000B08000212846F8F705FE00213846F8F7F2
:107F500001FEC2E1CCF1000001B2504200B2FBF7D9
:107F6000BDFD206026F85A8FB4F9020043F2046187
:107F70004143090C7180B4F90010084443F20461D4
:107F80004843000CB08000212846F8F7E3FD0021AB
:107F90003846F8F7DFFDF7E12846F8F765FE0123DC
:107FA0001A4605214DE019461046FBF797FD206063
:107FB000B4F9020043F204614143090C26F85A1F48
:107FC000A6F80280B4F90010084443F20461484363
:107FD000000CB08000212846F8F7BCFD002138468F
:107FE000F8F7B8FD25E2584201B2CCF1000000B22A
:107FF000FBF774FD2060B4F90200B4F9001043F2FD
:10800000046201445143090C26F85A1F05E019E2A5
:10801000BEE166E111E1B7E05FE05043A6F80280FF
:10802000000CB08000212846F8F794FD0021384666
:10803000F8F790FD5BE22846F8F716FE01231A4692
:1080400006213846F8F710FE01212846F8F782FD90
:1080500001213846F8F77EFDF84CF94D208928803B
:1080600060896880208AA8802846F9F73DFCB9F825
:108070005A10EA8848461144A9F86010B9F85C1013
:108080002A891144A9F86210B9F85E106A8911446E
:10809000A9F864102A7EA4F13401012A73D030F8C3
:1080A0005A2F0A8042884A80B9F85E008880E348E7
:1080B0000A882C3802804A88428089888180816AB7
:1080C000884794F8360000287ED0F8F7CBFF14F8E4
:1080D000360F401E2070BDE8F09F80461146604676
:1080E000FBF7FCFC2060B4F9020040F681514843E4
:1080F00081136180B4F9000040F68152504380132F
:108100000A18A2F681525242208052081144A9F85E
:108110005E204C46A9F85C10084424F85A0F002150
:108120002846F8F717FD00213846F8F713FD218897
:10813000A8F806106288A8F80820A388A8F80A30D2
:10814000C1F5586083B2B3F5227F02D9A8F80CA01C
:1081500015E08A1A92B24046A8F81620B2EB430FF7
:1081600001D96C3909E001F5227189B28181B1F53B
:10817000586F04D38670ABEB0101A8F80C100123F3
:108180001A460621C2E6B6E18046504201B2584284
:1081900000B2FBF7A3FC2060B4F9020040F6815165
:1081A000484380136080B4F9001040F68152514377
:1081B00089134218A2F681525242218052084C463D
:1081C000A9F85E20104400E09DE124F85A0F08440D
:1081D000608000212846F8F7BDFC00213846F8F7FA
:1081E000B9FC2288A8F806206088A8F80800A388AF
:1081F000A8F80A30C0F558618BB2B3F5227F02D9D6
:10820000A8F80CA015E0821A92B24146A8F81620F0
:10821000B2EB430F01D96C3809E000F5227080B24F
:108220008881B0F5586F04D38E70ABEB0000A8F8CE
:108230000C0001231A46052168E68046614618466F
:10824000FBF74CFC2060B4F9020040F68151484332
:1082500080136080B4F9001040F6815251438913B5
:1082600042182180A2F6815252424C46520824F80C
:108270005A2F1044A0800844608000212846F8F757
:1082800069FC00213846F8F765FC2188A8F806103B
:108290006088A8F80800C0F55861A2888BB2A8F8D9
:1082A0000A20B3F5227F02D9A8F80CA015E0821AA3
:1082B00092B24146A8F81620B2EB430F01D96C38B0
:1082C00009E000F5227080B28881B0F5586F04D3C0
:1082D0008E70ABEB0000A8F80C0001231A460721B2
:1082E0005AE68046CCF1000001B2504200B2FBF7E2
:1082F000F5FB2060B4F9020040F681514843801339
:108300006080B4F9001040F681525143891342183D
:108310002180A2F6815252424C46520824F85A2F2C
:10832000104460800844A08000212846F8F712FC21
:1083300000213846F8F70EFC2188A8F8061062885C
:10834000A8F80820A188A8F80A10C1F5586083B2DF
:10835000B3F5227F02D9A8F80CA015E08A1A92B2D0
:108360004046A8F81620B2EB430F01D96C3909E05A
:1083700001F5227189B28181B1F5586F04D38670FD
:10838000ABEB0101A8F80C1001231A46062103E605
:10839000804619461046FBF7A1FB2060B4F90200A5
:1083A00040F68151484380136080B4F9001040F6D4
:1083B0008152514389134218A2F6815252422180C0
:1083C00052084C46A9F85C20104424F85A0F08447F
:1083D000A08000212846F8F7BDFB00213846F8F7B9
:1083E000B9FB2288A8F806206188A8F80810A1889F
:1083F000A8F80A10C1F5586083B2B3F5227F02D9FC
:10840000A8F80CA015E08A1A92B24046A8F81620E7
:10841000B2EB430F01D96C3909E001F5227189B241
:108420008181B1F5586F04D38670ABEB0101A8F8D8
:108430000C1001231A460521FDE500006C00002008
:10844000940900208046584201B2CCF1000000B2ED
:10845000FBF744FB2060B4F9020040F68151484329
:1084600080136080B4F9001040F6815251438913A3
:108470004218A2F68152524221805208A9F85C208B
:108480001044A9F85E004C46084424F85A0F002115
:108490002846F8F75FFB00213846F8F75BFB218898
:1084A000A8F806106288A8F80820C1F55860A288CC
:1084B00083B2A8F80A20B3F5227F02D9A8F80CA04D
:1084C00015E08A1A92B24046A8F81620B2EB430F84
:1084D00001D96C3909E001F5227189B28181B1F5C8
:1084E000586F04D38670ABEB0101A8F80C10012380
:1084F0001A4607219FE530F8602F0A8042884A809B
:10850000B9F86400D2E505480088A0F5D041683983
:108510003FF4E1ADBDE8F05FF9F776BC182C0140FF
:108520002DE9F041904C9148B4F85A100288511A44
:1085300089B20F296FD30088A4F85A008C480088AC
:10854000DFF83082C0074FF000054FF0010741D03F
:10855000874AD4E90C1024321388B1EB530F02D2AE
:108560001288511A08444FF4F371884200D2084629
:108570008149B1FBF0F0616CC1F35101084406463A
:108580006064F7F74CFF00227C4BF7F7B4FE4FF026
:1085900040427B4BF7F7AFFE0E22F7F71BFFF7F7D2
:1085A00075FFA4F8A40094F86500401CC0B284F8DC
:1085B0006500082834D36C4898F84620001F0378DB
:1085C0009A4201D0027045806E4A13786E4A23B1F8
:1085D000458021E06564A56458E0D8F89410A1F5C1
:1085E000FA618E4211DD616D8B1C9E4205DDB0F992
:1085F00002100A290DDA491C06E08E4205DAB0F9AC
:108600000210002908DD491E4180B0F902000A2845
:1086100002DB177001E0A2E01570666584F8655012
:108620005A484FF4A5420178C1F38101012949D08C
:1086300002294AD044F687712181A4F8A020B0F91C
:10864000243089B24B439B13A4F89C30B0F90E0040
:1086500000237043B0FBF1F0A16CC0F3D100C1EB7B
:10866000C101C90200EB9130A064F017810341EA17
:108670009641B003F7F758FDB4F8A210C1EBC10161
:10868000C902C00800EB9130A4F8A200616CA06E92
:108690000844A06694F86C20521CD2B284F86C2076
:1086A000082A05D3C008A4F86E0084F86C50A566AB
:1086B000374A384ED388580633D498F80F0002282A
:1086C00006D02CE043F20451B6E744F24621B3E76A
:1086D000B06840F69916B04221DD94F8380094F85D
:1086E0008660B0420CD084F8860094F83D0000F01B
:1086F0000106C0F34000864202D1A4F8825004E093
:10870000B4F88200B0F5966F05D2B4F88200401C30
:10871000A4F8820005E043F08000D08001E0A4F8D6
:108720008250114894F83F20B0300C2A01D2C57411
:1087300000E0C774174B41F2482641F2504C93F8C1
:108740003C400C4B0C2AB3F882300AD3B14208DB10
:10875000012C06D0614502DD002B00D18774BDE8F5
:10876000F0818574FBE70000480100200407002029
:1087700000040040A40200204564BD0100209C408C
:10878000133B3340F2030020F3030020C004002019
:10879000140A0020280500202DE9F041384C394EFC
:1087A000394F207841F23331C2074FF000050CD029
:1087B000A28962B394F90700002800DA4042C0B2EF
:1087C000032829D240F2AE702AE0A570E5732F4A43
:1087D000E571A58192F83830237220F00800A1805D
:1087E00040F0020020703D867560B560F560916CC8
:1087F000490005D041F68461A18140F0100020704D
:10880000C0B240F0010020706574BDE8F081658160
:1088100020F01000207015E0042803D240F651002B
:1088200060810FE0052802D240F69910F8E740F683
:10883000CC42062803D3072801D3082801D262813D
:1088400000E0618197F89D0098B9B088102301B2CB
:10885000B4F90A003622FCF72FF87060F168401A6C
:10886000B1680844B060B6F900104843C013F06026
:108870003886388E10B10120A070C6E7A570C4E715
:108880001C0C002084060020A402002048010020C7
:108890002DE9F041554C2678F0077CD05448217AD8
:1088A000544D90F8380081427BD0534A2346DFF87C
:1088B0004CC1575C93F90E2093F90730874203D0DF
:1088C0001CF80170874213D146F002065B1C26702B
:1088D0005BB2E3711CF80110814201D15B1CE371B2
:1088E00094F90710062901DD0621E171521C1CE0F4
:1088F000434F17F801C0434F844503D017F801C018
:10890000844513D126F002065B1E26705BB2E3712C
:10891000795C814201D15B1EE37194F907306FF0FD
:1089200005018B4200DAE171521EA273207294F9A4
:1089300007108A1C042A02D941F68462A2812C4ABB
:10894000012912780ADD2B4B56079B6802D543F0AC
:10895000080301E023F00803AB606070B1F1FF3F52
:1089600009DA5107A96802D521F0080101E041F0B8
:108970000801A9606070F9F7EFFCA078012810D118
:1089800021488068A3280CDA94F90700022803DD47
:108990000220E07105E01EE06FF00101884200DA7C
:1089A000E171A089002630B1401E0004000CA081B6
:1089B00001D1E671A673E87B04280CD0B5F930101C
:1089C000512341220020FBF777FF2886002802D19F
:1089D000E07B10B1A670BDE8F0810C4806700C4831
:1089E0000670207820F001002070F4E71C0C0020B5
:1089F00048010020A40200202C96000832960008AE
:108A00003E9600084496000828050020180700201C
:108A1000FB060020B83ED93C223B8E391938BF36C0
:108A20007D35503436332D3234314830692F962E0F
:108A3000CE2D0F2D5A2C000000361C070038AA0A34
:108A4000003AAA0A003CCC0C003ECC0C0040380E88
:108A50000042380E0044380E0046380E0048380EEA
:108A6000004AC711004CC711004EC7110050C71172
:108A70000052C7110054C7110056C7110058C71142
:108A8000005AC711005CC711005EC7110060C71112
:108A90000062C7110064C7110066C7110068C711E2
:108AA000006A00000036000000388E03003A8E0392
:108AB000003CFA04003EFA0400401C0700421C0778
:108AC00000441C0700461C0700481C07004A880891
:108AD000004C8808004E880800508808005288081A
:108AE000005488080056880800588808005A8808EA
:108AF000005C8808005E88080060880800628808BA
:108B0000006488080066880800688808006A000019
:108B10000036000000388E03003A8E03003CFA0451
:108B2000003EFA0400401C0700421C0700441C07DA
:108B300000461C0700481C07004A8808004C8808AB
:108B4000004E8808005088080052880800548808A1
:108B50000056880800588808005A8808005C880871
:108B6000005E880800608808006288080064880841
:108B70000066880800688808006A0000003A22023F
:108B8000003C8E03003EB0050040D2070042AA0A16
:108B90000044CC0C0046EE0E00481111004A33137D
:108BA000004C9F14004E0B16005077170052771799
:108BB000005477170056771700587717005A771721
:108BC000005C7717005E77170060771700627717F1
:108BD000006477170066771700687717006A7717C1
:108BE000006C7717006E00000036000000388E031E
:108BF000003A8E03003CFA04003EFA0400401C07D1
:108C000000421C0700441C0700461C0700481C07C4
:108C1000004A8808004C8808004E880800508808E0
:108C200000528808005488080056880800588808B0
:108C3000005A8808005C8808005E88080060880880
:108C40000062880800648808006688080068880850
:108C5000006A0000003A2202003C8E03003EB0058C
:108C60000040D2070042AA0A0044CC0C0046EE0E97
:108C700000481111004A3313004C9F14004E0B168C
:108C80000050771700524F1A0054BB1B0056271D87
:108C90000058931E005A0020005C6C21005ED82210
:108CA000006044240062B0250064662600661C272C
:108CB00000681C27006A1C27006C1C27006E00003F
:108CC000003400000036000000380000003A0000C8
:108CD000003C0000003E0000004000000042000098
:108CE000004400000046000000480000004A000068
:108CF000004C0000004E0000005000000052000038
:108D0000005400000056000000580000005A000007
:108D1000005C0000005E00000060000000620000D7
:108D20000064000000660000006844145858587041
:108D3000111158585870411158584870111448581A
:108D400058701411584858703D1A0056E11A0054D2
:108D5000E11A0052851B0050281C004ECC1C004C10
:108D6000141E004AB81E00485C1F00460020004444
:108D7000A3200042EB2100403323003E7A24003C34
:108D80006626003AAE270038F5280036E12A00347E
:108D9000CC2C0032142E00305C2F002EA330002C7F
:108DA000EB31002A333300287A340026C235002400
:108DB0000A37002251380020E13A001E283C001CEE
:108DC000B83E001A00400018004000160040001491
:108DD00000400012004000100040000E0040000C57
:108DE0000040000A00400008004000060040000467
:108DF00000400002004000000102030405000500DD
:108E0000010203040104000305020000F001000058
:108E100036010000F8000000BA0000007C000000ED
:108E20007C0000007C000000411414111114441156
:108E3000141441110000290052007B00A400CC0052
:108E4000F5001E01470170019901C201EA011302F8
:108E50003C0265028E02B602DF02080330035903AA
:108E60008203AA03D303FB0324044C0475049D046A
:108E7000C504EE0416053E0567058F05B705DF0539
:108E800007062F0657067F06A706CE06F6061E071C
:108E900046076D079507BC07E4070B083208590819
:108EA0008108A808CF08F6081D0944096A09910934
:108EB000B809DE09050A2B0A520A780A9E0AC40A72
:108EC000EA0A100B360B5C0B820BA80BCD0BF30BD5
:108ED000180C3E0C630C880CAD0CD20CF70C1C0D5E
:108EE000410D650D8A0DAF0DD30DF70D1C0E400E13
:108EF000640E880EAC0ECF0EF30E170F3A0F5E0FF6
:108F0000810FA40FC70FEA0F0D103010531075100A
:108F10009810BA10DD10FF1021114311651187114F
:108F2000A911CA11EC110D122E12501271129212C7
:108F3000B312D412F4121513361356137613961374
:108F4000B713D713F6131614361456147514941455
:108F5000B414D314F214111530154E156D158C156B
:108F6000AA15C815E7150516231641165F167C16B7
:108F70009A16B716D516F2160F172C17491766173B
:108F80008317A017BC17D917F51711182E184A18F0
:108F9000661881189D18B918D418F0180B192619DD
:108FA00042195D1978199219AD19C819E219FD19FC
:108FB000171A311A4C1A661A801A991AB31ACD1A4E
:108FC000E61A001B191B331B4C1B651B7E1B971BD2
:108FD000AF1BC81BE11BF91B121C2A1C421C5A1C8C
:108FE000721C8A1CA21CBA1CD21CE91C011D181D73
:108FF000301D471D5E1D751D8C1DA31DBA1DD01D86
:10900000E71DFD1D141E2A1E401E571E6D1E831EC9
:10901000981EAE1EC41EDA1EEF1E051F1A1F2F1F3C
:10902000451F5A1F6F1F841F991FAE1FC21FD71FD6
:10903000EC1F002000006400C9002D019201F7011F
:109040005B02C00224038903ED035204B6041A052F
:109050007F05E3054706AB060F077307D7073B08F5
:109060009F0802096609C9092D0A900AF30A560BDE
:10907000B90B1C0C7F0CE20C440DA60D090E6B0EF7
:10908000CD0E2F0F900FF20F5310B4101511761153
:10909000D71138129812F8125813B81318147714FD
:1090A000D61435159415F3155116B0160E176B1707
:1090B000C91726188318E0183D199919F519511A7E
:1090C000AD1A081B631BBE1B181C731CCD1C261D70
:1090D000801DD91D321E8A1EE31E3B1F921FEA1FF0
:1090E00041209820EE2044219A21EF214522992207
:1090F000EE2242239623E9233C248F24E2243425C4
:109100008525D72528267826C82618276827B72733
:1091100006285428A228EF283D298929D629222A61
:109120006D2AB82A032B4D2B972BE12B2A2C722C5E
:10913000BB2C022D4A2D912DD72D1D2E632EA82E2E
:10914000EC2E302F742FB82FFA2F3D307F30C030E7
:10915000013141318131C13100323F327D32BA3289
:10916000F73234337033AC33E73322345C34953424
:10917000CE3407353F357735AE35E4351A365036BF
:109180008536B936ED36203753378637B737E93766
:10919000193849387938A838D738053932395F391C
:1091A0008B39B739E2390D3A373A603A893AB23AEF
:1091B000DA3A013B283B4E3B733B983BBD3BE03BDF
:1091C000043C263C483C6A3C8B3CAB3CCB3CEA3CF8
:1091D000093D273D443D613D7D3D993DB43DCE3D3A
:1091E000E83D013E1A3E323E493E603E763E8C3EB0
:1091F000A13EB53EC93EDC3EEF3E013F123F233F5C
:10920000333F433F513F603F6E3F7B3F873F933F3C
:109210009E3FA93FB33FBC3FC53FCD3FD53FDC3F5D
:10922000E23FE83FED3FF13FF53FF93FFB3FFD3FB8
:10923000FF3FFF3FFF3F0000E7382C35002020EFC5
:109240002037202333202620210000800200040044
:1092500008001000000200040008040000020004DE
:109260000008001000200040008004000000008082
:109270000000004000000020000000100000000876
:109280000000000400000002000000010000800057
:109290000000400000002000000010000000080056
:1092A0000000040000000200000001000080000037
:1092B00000080140000C0140000C0140000C01407E
:1092C000000C0140000C0140000C0140000C01406A
:1092D000001001400010014000100140001001404A
:1092E000001001400010014000100140001001403A
:1092F0000014014004080140040C0140040C01402A
:10930000040C0140040C0140040C0140040C014019
:10931000040C0140041001400410014004100140FD
:1093200004100140041001400410014004100140E9
:10933000041001400414014008080140080C0140D9
:10934000080C0140080C0140080C0140080C0140C9
:10935000080C0140080C01400810014008100140B1
:109360000810014008100140081001400810014099
:109370000810014008100140081401400C08014089
:109380000C0C01400C0C01400C0C01400C0C014079
:109390000C0C01400C0C01400C0C01400C10014065
:1093A0000C1001400C1001400C1001400C10014049
:1093B0000C1001400C1001400C1001400C14014035
:1093C00010080140100C0140100C0140100C01402D
:1093D000100C0140100C0140100C0140100C014019
:1093E00010100140101001401010014010100140F9
:1093F00010100140101001401010014010100140E9
:1094000010140140000000000000000000000000F7
:10941000000000000000000014080140140C01408E
:10942000140C0140140C0140140C0140140C0140B8
:10943000140C0140140C01401410014014100140A0
:109440001410014014100140141001401410014088
:1094500014100140141001401414014000000000D9
:1094600000000000000000000000000000000000FC
:10947000FFFFFF0F0FFFFFFFFFF0FFFFFF0FFFFFDB
:10948000FFFFF0FF0FFFFFFFFFF0FFFFFF0FFFFFEA
:10949000FFF0FFFF0FFFFFFFFFF0FFFFFF0FFFFFDA
:1094A000FFFFF0FFFFFF0FFFFFFFFFF0FFFFFF0FCA
:1094B000FFF0FFFF0000004040000000000400003B
:1094C0000040000000000400400000000004000014
:1094D0000040000000040000400000000004000004
:1094E00000400000000004000000400000000004F4
:1094F0000000004000040000000000808000000028
:10950000000800000080000000000800800000004B
:10951000000800000080000000080000800000003B
:10952000000800000080000000000800000080002B
:10953000000000080000008000080000000000207B
:1095400020000000000200000020000000000200D7
:1095500020000000000200000020000000020000C7
:1095600020000000000200000020000000000200B7
:1095700000002000000000020000002000020000A7
:1095800000000060600000000006000000600000B5
:1095900000000600600000000006000000600000FF
:1095A00000060000600000000006000000600000EF
:1095B00000000600000060000000000600000060DF
:1095C00000060000008002000400080010000002F5
:1095D000000400080400000200040008001000203D
:1095E0000040008004000000FF7FFFFFFDFFFFFF41
:1095F000FBFFFFFFF7FFFFFFEFFFFFFFFFFDFFFF99
:10960000FFFBFFFFFFF7FFFFFBFFFFFFFFFDFFFF7C
:10961000FFFBFFFFFFF7FFFFFFEFFFFFFFDFFFFF96
:10962000FFBFFFFFFF7FFFFFFBFFFFFF0102030400
:109630000500020304050001030405000102050002
:109640000102030404050001020355050010AA1AD3
:1096500055250030AA3A0000AA0A55150020AA2A6A
:109660005535FF3F84960008000000202C070000BD
:10967000E8060008789700082C070020B4090000CD
:10968000D863000845020406082D010203040405FE
:109690005006070809139D2B1B08B104211355150B
:1096A0002A40061908019713E93D14080D3E1B08CE
:1096B0000904012D17020604050103148020FF8B05
:1096C000AA0A02019C15AA0A551500085920AA2ABF
:1096D0005535FF3F072903010504060203127C15D7
:1096E00073FFFF04FF8080010125025B6402130AFF
:1096F00013456712081201100C050406020301014C
:1097000003070505280B01020304020607030304EF
:109710000C3D0706040509191F1919043105060631
:109720002FAA1A381EAA1A064902290C2902312E1C
:1097300040FD3969260211042F405F020C26405B70
:10974000262ACD55155515123902017F0316D0076B
:109750001AFF01013B0261AA6C080108A80916C49E
:1097600091220312100A17401C12600A16901B0166
:089770004913596702000800CB
:020000040800F2
:10FC00004A46545A594D46312D4E3330202020203B
:10FC1000050406020301AA0AAA0AAA0AAA0AAA0A4B
:10FC2000AA0ADE3F00100000FF0131000201664613
:10FC300000400040513800400040004000400101B9
:10FC400000400040FF387B257B257B25FF003333B8
:10FC50000201401F00016626B81E6626FFFFFFFF57
:10FC6000FFFF01010100010000000300000202008B
:04FC70000000AA5591
:04000005080000ED02
:00000001FF
